:020000041100E9
:103000007FB50023284C294D03932800217C284AB2
:1030100001F0D9FA002812D103232800217C03AA49
:1030200001F078FA00280AD1224B039A9A4206D17D
:10303000214B2248E360224B636104B070BD02263D
:10304000217CFE2228001F4B009601F035FA002853
:1030500001D00020F1E71C4BA2899A42F9D1217CD2
:10306000FF222800194B009601F026FA0028F0D123
:10307000E389174A934203D1164B17486361DCE793
:10308000164A9342E5D1164B164A1B68934206D95D
:10309000C02304222800217C9B0001F076FA124B09
:1030A00012486361C9E7C0469461FF1FD441FF1F06
:1030B000813700005959530059598320A4BA00118F
:1030C000F9410011A061FF1F59590000A261FF1FC3
:1030D00083050000AD41001184BA00118215000083
:1030E000B861FF1F87130000B542001194BA0011A8
:1030F000002370B51A4E1B4C30006361637401F0FD
:1031000089F9402323744B2B0CD9CC233821AC22D2
:1031100030009B01217401F038FA00280AD0002504
:1031200025740CE0FFF76CFF051E08D1237C0433E7
:10313000DBB2E7E70C4B0D4D63610D4BE381236878
:10314000002B08D1002D06D00C222900200008F009
:103150000BFC2B7B6374300001F09AF970BDC04604
:10316000D441FF1F9461FF1F4D42001174BA00113A
:10317000AAAAFFFFF7B5164B0192C318021D002043
:10318000009388235B05D3181B685C1C1AD09CB283
:10319000402C18D88D781E0CAC466746CD782D0291
:1031A0003D43AE4206D1019800280ED110000C70AC
:1031B000240A4C7003249BB20733A343D218009B0C
:1031C0009A42DED3FEBD4432F9E71000FAE7C0466A
:1031D000FC0F0000802213B503000324019189B283
:1031E000520107319B18A14304305A1A88235B050A
:1031F000C3181B68591C03D190429241104016BD60
:1032000099B2402907D80B000733A343C018904256
:10321000ECD30020F3E74430F9E7134B134A1B6863
:10322000126810B5FA24934201D81A00F824104B02
:10323000E4021B689A4210D813000E4A12689A42A0
:103240000ED3013307D1F823DB029C4203D10A4994
:10325000054808F089F9200010BDFC24E402ECE7E1
:10326000FE24E402F7E7C04600C0071100D00711B2
:1032700000E0071100F00711FFFFFF7FF0B59BB0E2
:10328000150004900391402A00D9A0E006AB5980B4
:103290001A80FFF7C2FF0400042816D9002206A9ED
:1032A000FFF768FF052810D906AB1B88AB420CD18D
:1032B000002D07D0514B2A000499C01808F074FA69
:1032C000002802D101201BB0F0BD06AB1D802000FC
:1032D0000699FFF77FFF041E7BD1069B0793FFF73C
:1032E0009CFF80235B01C618802307001B039E42BE
:1032F00001D3F826F60288235B05F31801931B68B7
:10330000013302D0019808F07FFA3D49019808F096
:103310002BF93B1D0293331D05938822029B520516
:103320009B181B6808935A1C3CD044219AB2009108
:10333000402A04D80320D11D814389B2009103990A
:103340001B0C8B4224D0402A22D80122300008A92D
:10335000FFF710FF021E1BD1380008A9FFF70AFF74
:103360000400042831D9009A059B9B188022520141
:10337000B218934240D288235B05C118009A09A86D
:1033800008F0F2FA1D4B009A09A9F01808F034FA77
:10339000009A029B9446634402931A4B029AFB18CC
:1033A0009A42BAD388235B05FC1821680198013939
:1033B00008F0DAF8200008F027FA039A07AB5A80E1
:1033C00030000799FFF706FF0400002C03D100200E
:1033D00079E70428FBD988235B05E018069908F0F3
:1033E000C3F80323EA1C9A4300D16BE7034B04990B
:1033F000E01808F001FA65E70424ECE70400001186
:10340000FFFFFF7FF80F0000F7B505001400402A0A
:1034100021D8002701AE71803780FFF7FEFE042817
:1034200016D93A003100FFF7A5FE042810D93688D6
:10343000BC420BD0BD4209D0221CB44200D9321C80
:10344000064B92B2C118280008F08EFA30B2FEBDC9
:10345000C04300B2FBE703204042F8E7040000113C
:1034600037B5042204000D0001A81649FFF7CCFF70
:10347000020004280BD1019BA34208D3AB4204D025
:10348000104901A80195FFF7F9FE01203EBD0E4C41
:1034900023682000019308F0B7F901992000013951
:1034A000019108F061F880235B01E418074B9C420E
:1034B000EED10422034901A80195FFF7DFFE0020A9
:1034C000E4E7C0465555000000C007110000081190
:1034D00030B589B008F078F910226946254807F020
:1034E0005BFF254B009A9A420ED1019B029A0F2B4B
:1034F00033D8002101240698013B08D2002900D0CE
:103500000292029B013331D10023029325E0551C26
:10351000F2D102002100EFE710341022200004A9AC
:1035200007F03AFF029B013301D1069B02938823E7
:1035300004995B05C918059B06981A03120B0491A0
:103540000592814203D02B4201D108F00DFA019B74
:10355000013B0193019B002BDED1029B002B03D08A
:10356000049304984168084709B030BDE025014C38
:103570002D03EFE700000111504859368022F8B5BD
:10358000964C974BD200002120001C6007F01CFFD6
:103590002300944A88331A60934B1A786A23002ACE
:1035A00000D01133E3620A232365904B37221B7846
:1035B0000820A3638E4B2118E361102323628D4BF7
:1035C0003B256361C823DB00A36123008C331A60B1
:1035D0002823013AE26320646364CA67043A211D28
:1035E000CA672100BC310D602100C0310860210094
:1035F000C4310B6021000635CC310D602100083D3F
:10360000C8310D602100D0310A602200D432106030
:103610002200D832136022000227E0322100176016
:103620004222DC310A6021001B3DE4310D602100A3
:10363000E83108602100EC310B6023000521F433F0
:1036400019602300F0331A602300183290331A6097
:1036500023009433186023001E3A98331A60AF2376
:10366000DB002360644BFA262363644B644DE36004
:10367000644BF031A3642300FF31FC33B600A1603A
:1036800021611E60A5627325E5656D3D6565A565D3
:1036900096255D4AAD00E264666258606766A5667D
:1036A00000270925A767E566584F594D6067200038
:1036B0002567E2673A6015279C30676007001A208B
:1036C00038602000A0300700212038602000A8309A
:1036D00007004C4838602000F83006602600642758
:1036E000A436376026005F3FAC3637602600033FC4
:1036F000B03637602600C637B4363760260000275C
:10370000B836376038269E60424E96205E64424E40
:103710005A66DE61414E9A645E62F53EFF3E9E62ED
:103720001E269A67354A8000DE661F675F67DD6583
:103730001D661862DA67BE23394A5B00E250394BD6
:10374000D838235004302250C4225200A350C6233C
:10375000E4205B00E1500433334AE1503349344BF9
:10376000D1603449800019503349E938FF38195085
:1037700032490430195032493248D161324911631B
:10378000324951631900F4310860CE2030494000BD
:1037900011603049195019002F48F83108602F493D
:1037A000D16582212E4A89005A501A002D490832CB
:1037B000D1671A002C49B432116088212B4A890044
:1037C0005A501A002A49883211602A4ADA6407F0EE
:1037D0006BFF012007F0C0FFF8BDC0460004FF1FCB
:1037E0003064FF1F006FFF1F0444FF1F4A0AFF1FC2
:1037F0003A07000080C3C9019A020000DC050000FE
:103800006A18000050C3000088130000F009FF1F71
:10381000204E00006509FF1F68100000C409000069
:1038200040420F0010270000FC00FF1F751CFF1F07
:103830000000FF1FC92CFF1F5130FF1FE92EFF1F83
:103840003520FF1F2527FF1F5120FF1FFD21FF1FD0
:10385000C11FFF1F4929FF1F312AFF1F8D19FF1F9D
:103860005528FF1F7925FF1F8525FF1FC11EFF1F3C
:10387000791FFF1F391EFF1F0223F0B50124644D7D
:10388000644E2B70644B91B01C70644F039333688B
:1038900000210820BB7006F059FC082006F050FB00
:1038A0000023984205D0BA78552A02D0332A00D096
:1038B000A1E03360042006F0C3FD07F095FEFFF79A
:1038C0005DFE07F0D9FD1F2201240021544B10AEEC
:1038D0001A70544B1C70544B1970544B1968914317
:1038E000163A0A431A60602219689143403A0A4323
:1038F0001A6007F0A1FD07F0EFFD4D4B9847C1207E
:10390000FF214C4B80001A588A431A50C52292005E
:1039100098588843BF390143995098584649084000
:103920008021C9010143802099509958C00509029E
:10393000090A0143995080214048490107F0ACFE33
:10394000032322003E49019400933E4807F09CFE69
:103950002C223D4905A808F007F805AC61782078CD
:10396000023406F00DFBA642F8D1384C01210020AC
:1039700006F01AFC0920012106F016FC2268344BDF
:1039800003201A40A023DB02134323608023226814
:103990009B041343236022682E4B1A4080239B0311
:1039A000134323602C4A2D4B934200D8012007F08B
:1039B0002BFD07F019FF80232268DB0413432360EB
:1039C000287807F0D1FE039B1878C0B207F07CFD81
:1039D00007F082FE2249042007F0CEFE06F0FCFC30
:1039E00000F040F800F008FE00F0B0FE00F00CFA25
:1039F000002011B0F0BD00932100194A042007F007
:103A00005BFE8023DB059C62FFF762FD52E7C04648
:103A10004A0AFF1F34F000400444FF1FC461FF1F27
:103A2000480AFF1F490AFF1F680AFF1FBCF0004039
:103A3000E1A2000000E100E0FF00FFFF0844FF1FDB
:103A40008C56FF1F0854FF1F98B9001114F0004056
:103A5000FF7FF8FFFFFF9FFF0080FF1F006FFF1F2A
:103A60003B000108002210B51100112007F024FDD1
:103A700010BD0000F8B500230926374F374C3B62D4
:103A8000E3681120B343E36007F016FF112007F04D
:103A900093FD112007F050FF402322688025134337
:103AA000236080236268DB0213436360A3682C4AAF
:103AB0002B43A360A36802211340A3608023A26864
:103AC0009B0113431022A360236C072093432364BC
:103AD000236C0F3A1343236480235B003B62226B09
:103AE000204B1A402263626B1A406263A26B1A4039
:103AF000A263E26B1340E363E3681B4A1340E36095
:103B000006F03EFA0121072006F04EFB174B11206C
:103B10005A6C15435D6407F077FDFD21144B154A7F
:103B200089005A508023C720626B5B031343636391
:103B3000E36880003343E3600F4B104A195811408B
:103B4000802212020A431A50802292051A6008222B
:103B50000B4B5A63F8BDC04600F000403CF00040FB
:103B6000FFFFDFFFEFFFEFFFFFFF7FFF00380040A9
:103B70000000FF1F5118FF1F00E100E0FF00FFFFE2
:103B80000000054070B5284C238C002B23D0228ADE
:103B9000002A21D1DA0023826382A382E382238375
:103BA0006383A383E38322606260A260E2601F4DAF
:103BB0001F4A6420EB8093420AD8FA220020D200E8
:103BC000934205D91B4A0A21981807F02DFCC0B270
:103BD00000232872238470BD0720E11CCA7F0132B4
:103BE0000240CA7705D10325201DC17F013129403C
:103BF000C17708325200A352002321001A00088A1C
:103C000001321B180231082AF9D1221DD27F9200FD
:103C1000A350626823689B18A2689B18E2689B18EF
:103C20005B099BB2C3E7C0460461FF1FAC61FF1F85
:103C3000B70B000030F8FFFF30B503A804880B2055
:103C4000002C0ED14968074D0878497809020143D4
:103C50000A20A94205D1012120001980024B1B7ABC
:103C6000137030BD192A0000AC61FF1FF7B51500B5
:103C700008AA16884A680F4F147852781202224315
:103C80000A24BA4214D10122DBB2019200962A0022
:103C900007F0F2FA041E0BD1074B1B68002B07D06C
:103CA00068782A7800021043424250410130984718
:103CB0002000FEBD022900003061FF1F30B5012544
:103CC00003790400BFB02B4211D00A49408806F0A6
:103CD0003FFE28420BD0084B01A95B8D4D800B8025
:103CE000064B00221B7A60880B7103F011FF3FB076
:103CF00030BDC0462861FF1F4840FF1FAC61FF1F59
:103D000010B50549054806F0D9FD0421044A0548C7
:103D100006F096FD10BDC0462861FF1FFFFF0000A2
:103D2000C4B900114840FF1F10B5024804F072FDED
:103D300010BDC046BD3C0011012303700B4B1A7A25
:103D40004270022282709A78C270DA78027103227D
:103D500042711A7982715A79C2710C2202729A796F
:103D60004272DB7983720B207047C046AC61FF1F43
:103D7000022310B50370013B437005338370103389
:103D80000371443B43712A3383714433C37100236D
:103D90000372064B04001B8843720A30FFF7CCFF06
:103DA000831D0A30C0B2E37010BDC046AC61FF1F76
:103DB00010B5142007F098FB124B14220021186054
:103DC00007F002FB002007F0A7FD012007F04CFBE5
:103DD000022007F031FD032003F0C0FF042005F0AE
:103DE000D5FF052003F0FEF9062003F0CBFE0720E7
:103DF00001F062FA082006F003FD092001F034F812
:103E000010BDC0463461FF1F07F0B6FB012007F06C
:103E10009BFB07F0B9FC0000094B10B50400984269
:103E200005D0012904D12000064906F047FD10BD48
:103E30000229FCD1013904F0ABFC0028F3D0F6E7ED
:103E4000FEFF00005A61FF1F70B50D7A100004AA32
:103E50002C00168810221440154220D1002E20D1AB
:103E60000A78022A18D14A68517815780E4A090250
:103E70002943914205D00D4A914209D01C800A2461
:103E800004E014220A491A8007F06EFD200070BD7C
:103E90000C2208491A80F7E71C800124F6E7082461
:103EA000F4E70B24F2E7C046F3FF0000F4FF000044
:103EB0009042FF1FC0BA001110B50400074908481E
:103EC00006F0FCFC074804F0E5FB0020E40704D5FD
:103ED0000721054A054806F0B3FC10BD5A61FF1FD3
:103EE000FFFF0000193E001108BA00118C40FF1FAF
:103EF00000B50C4BBFB01A780B4902A800F0E0FCEB
:103F00006B4680B2D880002809D06A46074B01A9C9
:103F10001B889380064B0022188803F0F9FD3FB000
:103F200000BDC0463861FF1F3961FF1FE640FF1F1B
:103F3000F041FF1F00B50C4BBFB01A780B4902A827
:103F400001F02CFD6B4680B2D880002809D06A466B
:103F5000074B01A95B8D9380064B0022188803F064
:103F6000D7FD3FB000BDC0466261FF1F6361FF1F08
:103F70008C40FF1FF041FF1FF7B50E00377A1C0081
:103F800008AB11003D001A8820231D401F423CD180
:103F90003378022B3BD173681F785B781B023B435D
:103FA0001E4FBB4208D01E4FBB4214D01D4DAB422A
:103FB00021D00A252800FEBD002A2AD1142C2AD897
:103FC0002200F06807F0D0FC174B1C70012CF1D9CF
:103FD000FFF7B0FFEEE7002A1BD1202C1BD82200F0
:103FE000F06807F0C1FC114B04211C70104B1878CD
:103FF00007F0B2F9DEE7E3B20124009201940A006F
:10400000310007F039F90500D4E70825D2E701258A
:10401000D0E70B25CEE70D25CCE7C046F3FF000027
:10402000F4FF0000022900006261FF1F3861FF1FDA
:10403000E461FF1F332310B5040003700A2207490F
:10404000013007F091FC064B0F201B681A0AE3723F
:1040500022731A0C1B0E6273A37310BDAC61FF1F99
:10406000D461FF1F30B5012503790400BFB02B4296
:1040700013D00B49408806F06BFC28420DD06A46ED
:10408000084B02A81B889380FFF7D4FF6B46D880AB
:104090000022608801A903F03BFD3FB030BDC0465F
:1040A0005A61FF1FE640FF1F10B5024804F0B2FB43
:1040B00010BDC0466540001170B5160004AA1488F2
:1040C00005AA15784A685078117800022A4A0843F0
:1040D000801805284BD807F0A7FB03131E29343F8F
:1040E0000720042C0BD80522121BAA4200D92A0053
:1040F00022491A803000091907F036FC002070BDF3
:104100000720112CFBD81222121BAA4200D92A0028
:104110001B491A80EEE707200E2CF0D80F22121B45
:10412000AA4200D92A0017491A80E3E70720032C86
:10413000E5D80422121BAA4200D92A0012491A808B
:10414000D8E70720032CDAD80422121BAA4200D990
:104150002A000E491A80CDE70720032CCFD804226D
:10416000121BAA4200D92A0009491A80C2E700227C
:104170000A201A80C3E7C046DCD5FFFF53BA0011FE
:104180008061FF1F43BA00113EBA001139BA001115
:1041900034BA001110B50D21024A034806F050FB55
:1041A00010BDC04628BA0011FC40FF1F13B5104CCB
:1041B0000423217C01AA00F0ADF9002815D16B463B
:1041C0009A88236852BA92B25343228909491B0C38
:1041D0009B184B806B46DA88636852BA92B253439D
:1041E00062891B0C9B188B8016BD0120FCE7C04622
:1041F0009461FF1FAC61FF1F13B5124C06236A4682
:10420000217C00F087F9002819D16B4619882368B2
:1042100049BA89B24B4321890B4A1B0C5B18538066
:104220006B46D97803335B781B020B435BBA61683A
:104230009BB24B4361891B0C5B18938016BD012018
:10424000FCE7C0469461FF1FAC61FF1F37B5174CF8
:1042500007236A46217C00F05DF9002824D16B46D3
:104260001B787F2B20D86B46DD78F0232A041B03B4
:104270001A406B469B880E495BBA9BB21A4323686F
:104280002D09534322891B0C9B184B806B465A788F
:104290009B7812031B011A4363682A4353436289C4
:1042A0001B0C9B188B803EBD0120FCE79461FF1F17
:1042B000AC61FF1F7FB50226154C0022217C03ABA9
:1042C0000096050000F0F8F8002802D0012004B0A4
:1042D00070BD0E23217C0122280000966B4400F063
:1042E000EBF80028F2D16B469A892368D2BA53437F
:1042F000228908491B149B184B806B46DA89636836
:1043000052BA92B2534362891B0C9B188B80DEE732
:104310009461FF1FAC61FF1F70B5184C237C002B0C
:104320000FD0382B0ED1164D280000F073F8CC2397
:10433000AC222800217C9B0100F027F9280000F026
:10434000A7F870BDE3890F4A934209D10C4D2800AC
:1043500000F060F800222800217C00F005F9EDE76C
:10436000094A9342EDD1064D280000F053F89022FF
:104370002800217C920100F026F9DFE79461FF1FFD
:10438000D441FF1F830500008320000070B5144C4A
:10439000237C002B1FD06369002B1CD0114D2800FB
:1043A00000F038F86369280098470400280000F0FE
:1043B0006FF8002C10D10C4B0422995E002905DA0D
:1043C0009C801A8801321A80200070BD074A9142F1
:1043D000F7DD9A80F5E70124FEF78AFEF4E7C04690
:1043E0009461FF1FD441FF1FAC61FF1F0F27000026
:1043F00010B58024064AA4001168436B234205D1FE
:1044000013685B1A032BF8D9012010BD0020FCE7CC
:104410006008FF1F70B5C17905000C00631E9C4148
:104420001A4BE402E41849000460C9B2007905F0AF
:10443000F1FEE979687949000131C9B205F0EAFE77
:10444000E8790930C0B207F077FA0023E3666133F8
:104450002360AA795B3B002A0ED022689A43023B74
:10446000134323600A23E36107332362002323639A
:10447000A3630133E36370BD22689A4302231343AD
:104480002360462363610633A361EFE700500040D9
:1044900070B5002504000368DD66C0790930C0B23C
:1044A00007F00AFA2900207905F050FE290060790A
:1044B00005F04CFE70BD0000F8B51E0006AB1D787F
:1044C000002304681700E366616007F07DF90123AB
:1044D0008022E3662B0027615200013B08D207F0DF
:1044E00013F908200A4A1168002D03D12800F8BDED
:1044F0002261F2E7236F034203D02369013D337049
:10450000013613685B1A032BEED90125EEE7C0468E
:104510006008FF1F70B51C00002305681600EB66DD
:10452000696007F051F901238022EB6623005200F5
:10453000013B08D207F0E8F808200A4A1168002C6D
:1045400003D1200070BD2A61F2E72B6F034203D034
:104550002B69013C3370013613685B1A032BEED9CB
:104560000124EEE76008FF1F002370B50468150002
:10457000E366616007F028F90123E366256107F02F
:10458000C3F82000FFF734FF70BD70B51D00002395
:1045900004681600E366616007F016F90123E3661C
:1045A00026610F33626B1A42FCD02B0A2361102361
:1045B000626B1A42FCD0EDB2256107F0A5F820002D
:1045C000FFF716FF70BD002370B504681500E366A1
:1045D000616007F0F9F80123E3662B0A23611023D9
:1045E000626B1A42FCD0EDB2256107F08DF8200015
:1045F000FFF7FEFE70BD000010B5084CE368002B0D
:1046000008D18022064B52021B689B186360054B41
:104610001B68236007F040F9A06010BDD461FF1F44
:10462000C8F00040CCF0004070B5184A936A916A17
:104630009942FBD116498A689A421FD39A1A8B6015
:10464000144B0126186893B2D202D20E4343424360
:1046500000204C681B0A1B1912029B180E4C0A689A
:104660004B60551CA3420CD8002801D04B600A6057
:104670000A4A136008680A4B186070BD581E821AF7
:10468000DDE7084A30009B182A00EAE700F0004006
:10469000D461FF1F140AFF1F40420F00C8F0004002
:1046A000CCF00040C0BDF0FF70B51F4C23793F2B0C
:1046B00001D93F2323711D4B22791A701878C0B29B
:1046C00006F0B2FF18231A491A4A0B801A491380C0
:1046D0000B805380A379194980200B800C21938093
:1046E00001334B43164D191C0001834200D9011CB4
:1046F0002980D1806379002B11D101336371237A32
:10470000012B01D8022323726279237A0D48534387
:104710000A21584306F088FE0B4D286070BDA02B7F
:10472000EDD9A023EAE7C046C861FF1F480AFF1F72
:10473000EE41FF1FB043FF1FEC41FF1FEA41FF1F87
:10474000E841FF1F71020000B861FF1FF8B5192191
:104750000020FEF785FE114C011E114D09D10C22DF
:10476000104BC1CBC1C4280006F02EFEFFF79CFF02
:10477000F8BD0C2220000C49FEF746FE0C2802D0A2
:10478000084B43CB43C40C2228000849FEF73CFEEB
:104790000C28EBD00C220021E5E7C046C861FF1FC2
:1047A0009461FF1FB4BA0011FC0C0000F50C00006E
:1047B000F0B51D4C8022A5440400882069465201B2
:1047C000400507F0A1F8902212016A44130020006E
:1047D00032C832C316C816C38023144C144FA668BF
:1047E0009B033343A3603B6006F0AEFD8823A068C3
:1047F0005B05C01807F008F80025882329008022EF
:10480000A0685B05C01840196944520006F0F4FF27
:1048100080230135FF355B019D42EED1A6603E60ED
:10482000044B9D44F0BDC046FCEFFFFF2043FF1F3B
:104830009808FF1F04100000F0B5040087B000289E
:1048400025D0684606F098FD1B4C022806D10622AA
:104850006946200006F0A8FF002816D0694600230C
:1048600001250F262F00E25C01331009103087402C
:1048700038002F00324097403A0002434A61043921
:10488000062BEFD16846FFF793FF07B0F0BD182263
:1048900069460A4807F038F86A46A300D35801333E
:1048A00005D01822FF21684606F08EFDEAE70134A4
:1048B000062CF1D1E9E7C0466509FF1F0009001188
:1048C000F0B5002504000E0085B0AA4200D183E0B7
:1048D0004B1C087801934B78897837790902194382
:1048E000F3783F061B040B431F430397207065704A
:1048F000252800D193E033D8112813D806F0B4FF4F
:1049000066000D010D010D010D01A700B500AE00FF
:104910000D010D010D010D010D010D010D010D0127
:10492000E7000701232800D1C0E0DB2800D016E112
:10493000042A00D8A9E01025052A05D0551F2A0011
:104940003800711D07F010F805223100200007F033
:104950000BF82A003900601D07F006F805353BE02A
:10496000562856D010D8332800D19AE0552836D092
:104970002628DAD1894B2900132218001D0006F0E1
:1049800023FDFEF7B5FB59E0712800D174E07228D1
:1049900000D17DE0DC28C8D1022A00D875E0737808
:1049A000BFB26370B378A370032A05D0033A39000D
:1049B00092B2F01CFEF762FC10223900E01CFEF7F8
:1049C00023FDC51C002807DA60705CE00C22200083
:1049D000734906F0C9FF0C25280005B0F0BD013A67
:1049E000704D0C2A13D8002A0AD02800019906F02D
:1049F000BBFFFFF759FE0C2228006B49FEF73EFC77
:104A000029000C22601C06F0AFFF0D25E4E70C2204
:104A1000EBE7644D654B2A0043CB43C2E9E7013A1B
:104A20005E4D0C2A11D8002A08D00199280006F002
:104A30009BFF0C2228005E49FEF720FC2900132270
:104A4000601C06F091FF1425C6E70C22EDE7062254
:104A50005849601C06F088FF0625BDE7122256491A
:104A6000601C06F081FF1325B6E708225349601C3D
:104A700006F07AFF0925AFE77178F02905D8504B89
:104A8000188801F0E7FB0225A6E7FF236370FAE729
:104A90004C4B012A03D072785A706270F3E75B784E
:104AA000F4E72000FFF7C6FA050095E7042A04D9C9
:104AB000454D2F6006F0F0FEA860FFF7B5FD04221B
:104AC000039003A9601C06F04FFF052584E73F4DC6
:104AD000062A15D906222800019906F065FE00284D
:104AE0000ED006220199280006F03EFF0622384922
:104AF0002800FEF7C3FB0123324A51780B43537061
:104B000029000622601C06F02FFF072564E7012A12
:104B1000BBD07078FFF790FEB5E7012800D004E71E
:104B2000931E2C4F132B06D87378002B0BD100F05B
:104B300009F900F03FF9284B39001D78601C6A1E06
:104B400006F012FF48E7551E2A000199380006F0CA
:104B50000BFF38002149AAB2FEF790FBE9E7DA28FB
:104B600093D1042A91D9082A15D9B37972791B02F5
:104B70001343F27912041A43337A1B0613433B6042
:104B80003B68052231002000039306F0EDFE04226D
:104B9000601D03A96CE7FE236370F1E79461FF1FBA
:104BA000C0BA0011C861FF1FFC0C0000B4BA0011AC
:104BB000F50C0000A061FF1F8061FF1F2443FF1F51
:104BC000F041FF1FC461FF1FD461FF1F6509FF1F74
:104BD000ADAC0000C563FF1FC363FF1FAEDE000066
:104BE00070470000020010B5094B0A32094C92B21E
:104BF000DA815A8298811882207802F091F9042291
:104C0000054B012120781A7006F0A6FB10BDC046A6
:104C1000AE42FF1F0E64FF1F0D64FF1F013870B509
:104C2000042809D806F000FE0309230812001E4BD1
:104C30000221187806F090FB70BD1B4B08211878F4
:104C400006F0FAFC0022194B1A72F5E780220024C4
:104C5000164B154D52001A81082128781A68DC720B
:104C600006F0C2FB2100287806F0B6FCE4E70E4B04
:104C70000821187806F0E0FC0D48FFF779F80D4B95
:104C80000D4A9B7993800D4A13800022074BDA72FC
:104C90000132FF321A810A4B5B78002BCCD0094AD3
:104CA000136006F071FBC7E7E461FF1FB861FF1FE7
:104CB000F941FF1FC861FF1FB043FF1FEA41FF1FFB
:104CC000C461FF1F34F0004010B5002905D1082849
:104CD00003D10131013005F067FA10BD10B501298B
:104CE0000FD108280DD10021013005F05DFA054BE8
:104CF0001B78002B05D02622034B04485A72FFF77D
:104D000071FF10BDE663FF1FB861FF1FC4090000FB
:104D10000300F0B50A4D8E18B14202D1520080183E
:104D2000F0BD0C782F6824093C5D0F271C700C78AF
:104D300001313C402F683C5D5C700233ECE7C046BB
:104D4000E441FF1F0E22124B10B51A700D23114CB7
:104D500011492370093A043B1048637006F004FEC1
:104D60002D2301220E490F48E371FFF7D1FF0122E5
:104D70000D49FFF7CDFF01220C49FFF7C9FF0300E2
:104D800000200B4902001870FEF778FA10BDC046EB
:104D9000E263FF1FC363FF1F53BA0011C563FF1F08
:104DA0006709FF1FCB63FF1F6609FF1F6509FF1F10
:104DB000AEDE000070B5134C142220001249FEF73D
:104DC00023FB431E114D132B19D8AB78002B16D0A3
:104DD000431C2B7009236B70002300190370287883
:104DE0000B4B01302900C0B2187006F0A5FC2978E1
:104DF00022000139C9B2002005F040FC70BDFFF768
:104E0000A1FFECE7C563FF1FAEDE0000C363FF1F19
:104E1000E263FF1F10B5114B1A781870002A0ED0EC
:104E200000280BD10E4B1A78062A07D85423D340FA
:104E3000DB0703D50B4B187802F072F810BD002881
:104E4000FCD0074B1B78012B02D0033B022BF5D87B
:104E5000044B0121187806F07FFAEFE7E663FF1FA5
:104E60000D64FF1F0E64FF1F70B5504E504A51492C
:104E70003070082005F08EFA0121092005F094F920
:104E8000092005F075FA0121002005F08DF90020B8
:104E900005F06EFAFEF72CF906F07EFB0322464978
:104EA0004648FFF735FF2D24030004221C704449B7
:104EB0000130FFF72DFF30230470424D424C437008
:104EC00083702E3B062220004049EB87FEF79CFAB8
:104ED000062813D0200006F04FFA022809D003213B
:104EE000200006F0D1FC8D23E3706E3B2371193353
:104EF0006371062220003549FEF7C0F9344B1B6868
:104F0000FC335C64FFF756FF0020FFF783FF314C52
:104F1000314A0121314B1278207801F0C3FF304A29
:104F2000304B12780021207801F0BCFF01222E4B7B
:104F30001A702E4B9B78552B31D12D4B3B325A7228
:104F40002C4B2D4AAB81EA812B826A82202130785A
:104F500006F092FC0120404205F0DCFB01204042BB
:104F600005F078FCFFF716F9FEF7CAFE00F0AEFC7C
:104F700001204042FEF7A0FF012006F065FCF02072
:104F800001F04CF90121307806F0E6F9307802F0B2
:104F900023F91A4806F0A8FCFEF76CFD70BD6422E8
:104FA000174B5B7953431A000A32CBE7E461FF1FCA
:104FB000C94C0011DD4C00112443FF1F8061FF1F0D
:104FC000A061FF1FAE42FF1F6509FF1FADAC0000CF
:104FD0003064FF1F0E64FF1F1842FF1FF941FF1FBF
:104FE000E263FF1FC363FF1FB463FF1FC461FF1FA2
:104FF000B861FF1FC4090000CE090000E661FF1F71
:10500000C861FF1FF8B50A0020230D001A4019429D
:105010005DD05C4B1B78002B42D0FFF705FB5A4B51
:105020005A4C5B4E99686268737A8A1ADB039A421B
:1050300002D36160FEF71EFD327A217A531EDBB285
:10504000994230D1FFF768F9637A002B25D0013BF4
:10505000DBB26372002B20D14E4B9B78552B01D1D4
:1050600006F092F9E37A002B12D00023A27AE372C1
:105070009A4202D0A372FEF785FD474A474F138834
:10508000380001331380FEF773FE390006F08CFA06
:10509000642370795843FFF7A5FD237A0133237207
:1050A00020206840F8BD9142CED300272772FFF739
:1050B0006DF9A37ABB4202D0A772FEF763FD374FAA
:1050C0003800FEF755FE390006F06EFABCE70BB269
:1050D000002B0ADA324B187806F04EFC002801D07B
:1050E00006F01AFB80200002DBE70224214206D0F2
:1050F000264B01201A72FFF78DFE2000D1E70B0727
:105100001BD5FFF791FA204B2049214C98684A683B
:10511000637A821ADB039A4202D34860FEF7AAFC44
:10512000FFF734F9FFF7F8F800F0EAFB2368DB0734
:1051300001D5FEF7B9FF0820B3E710230E001E408B
:10514000194209D0FEF71EFD0E4B1B78002B01D132
:10515000FEF7EAFD1020A4E70124214209D01148FE
:1051600000F06EF806F078FA3100092005F01CF81E
:10517000C3E7042408002040214200D192E7FEF753
:10518000B7FEBAE7E663FF1FD461FF1FB861FF1FD8
:10519000C861FF1FC461FF1FAC61FF1FF941FF1F02
:1051A000E461FF1FDC41FF1FF0B51B4B1B4F1B8849
:1051B0003A8804001A4E1B4D85B09A420DD83288A9
:1051C0009A420AD3184B1A882B889A4205D1174A5B
:1051D000174B12881B889A421BD0052001F074F8E7
:1051E0003B8802AA13803388019053802B88114D8D
:1051F00093800F4B02A91B88D3800F4B2A78188805
:1052000002F090FD0D4B08212878019A1C7006F0E1
:10521000A3F905B0F0BDC046B263FF1FEE41FF1F0A
:10522000EC41FF1FEA41FF1FB063FF1FAE63FF1F8A
:10523000E841FF1F0E64FF1FF041FF1FAC63FF1F1B
:1052400013B50C4B1C78002C11D1002801D00A4B4F
:1052500018600A4A0A4B11780A4A10780A4A0192E1
:105260000A4A0092002205F001F9200016BD11241F
:10527000FBE7C0460D64FF1FA863FF1F0C64FF1F00
:10528000FC63FF1F0E64FF1FE863FF1FEC63FF1F3B
:1052900010B5064B12201B78052B06D1044B1322A8
:1052A0001988044B187801F0EBF910BD0D64FF1F4D
:1052B000F041FF1F0E64FF1F10B500240122114BA7
:1052C00052421870104B1C70104B1A8001F084FF72
:1052D00004220F4B21001A700E480C3206F05CFAC3
:1052E000102221000C4806F057FA07220B4B1C60D5
:1052F0000B4B1C700B4B1C700B4B1A700B4B1C7028
:1053000010BDC0460E64FF1F0D64FF1FF041FF1F5C
:105310000C64FF1FFC63FF1FEC63FF1FE863FF1FAC
:10532000C263FF1FC163FF1FF241FF1FC063FF1F66
:10533000F8B5174C0600257806A814240078052D2A
:1053400023D1B41F134FA5B21824BD421DD88D1F01
:10535000ADB2BD4219D8FA256D00AA4215D21D0082
:105360000D4F0A3DADB2BD420FD80C4C26800C4CFF
:1053700021800C4900240A800B4A1380FFF714FF98
:105380000A4B0421187806F057F92000F8BDC046F2
:105390000D64FF1F790C0000750C0000EE41FF1F2B
:1053A000EC41FF1FEA41FF1FE841FF1F0E64FF1F92
:1053B000F0B50BB20D0089B0002B00DB70E1A44EFC
:1053C000307806F0D9FA041E50D00378A22B00D111
:1053D00022E1D02B1AD0912B45D143780E2B42D10C
:1053E0009C4B82889A423ED19B4A83681278052A58
:1053F00039D1032018567F2835D0984B1B68002BD5
:1054000031D05B68002B2ED098472CE0807807289D
:1054100029D806F009FA0428183F3F74A8D8637801
:10542000002B0CD101218C4B19708D4B1A78002A5E
:105430005BD08C4B307801F035FD002855D0072229
:10544000854B1A7051E061780029F8D1E378002B80
:1054500011D0854A854B1278307801F023FD6070B9
:105460006378002BEBD1200006F056F98020000273
:10547000684009B0F0BD784B1B78022BF3D00121B6
:10548000307806F041F80028EAD10121307805F0A3
:1054900063FFE5E76378002BD1D16F4F032807D175
:1054A0003B78052B02D101333B701EE00223FBE762
:1054B0006F4B1A886F4B0293002A0BD01B78002B7E
:1054C00003D00121307806F047F83B78062B04D151
:1054D000013BE9E7029B1A70F7E7042B41D1012158
:1054E000029B3078197005F037FF5C4B1B68002B6E
:1054F000B9D01B68002BB6D0574A107884E7637880
:10550000554F002B27D10622211D5B4806F02CFAAF
:1055100062895A4B5A491A80A2895A4B1A80E389E8
:105520000B800521397058490A80584A1380228A15
:10553000574B1A80574B1B78012B09D11F2000F0C5
:10554000C3FEFA22920042430421307806F004F8A8
:105550000022484B75E7312B00D070E70022454B05
:105560001A700323A0E706220021434806F014F92D
:105570000023454A04211380444A30781380444A6A
:10558000138006F059F80821307806F055F8A37911
:10559000083B5A425341304A03331370304B1B7857
:1055A000002B06D0334B30781A78002A06D001F051
:1055B000B7FC0122314B52421A8096E70121197043
:1055C00005F0CAFEF5E70821307806F035F8637873
:1055D000002B00D047E72C4B2D4F0293E388029A13
:1055E00004211380294B307803932389039A138075
:1055F00063893B8005F088FF002800D033E7264B05
:105600001B68002B00D12EE7039902983A8809887D
:1056100000881B68984726E74379132B00D022E7C0
:105620000389012B0AD11D4B1B78022B06D10821BF
:10563000307806F001F8FFF72BFE14E7052000F0A4
:1056400043FE08210200307805F086FF0BE7C046D4
:105650000E64FF1F051400000D64FF1FA863FF1FE9
:105660001842FF1FF941FF1FE263FF1FC363FF1FC3
:10567000E463FF1FE663FF1FB563FF1FF041FF1FD9
:10568000BC63FF1FBE63FF1FB263FF1FB063FF1F3A
:10569000AE63FF1FB463FF1FA463FF1FAC63FF1F54
:1056A0008020C001014200D0E2E6CB0731D5324B69
:1056B0001B78002B1DD0314E05AC3378052B1AD149
:1056C000023B23702E4B21001B7823722D4B1B783D
:1056D00063722D4B187801F089FB002809D0072050
:1056E0002A4B30701B68002B03D01B68002B00D0A6
:1056F00098470120BCE60E20254B06221B78254941
:105700002370254B1B78637002ABC01806F02CF990
:10571000D8E7022308001840194209D0174B1B781C
:10572000052B03D11D4B188805F0CEFF02209FE604
:105730000424214203D0FFF737FD200098E6082318
:1057400008001840194200D193E6154B1C78012C33
:1057500003D0022C0DD008208AE6124B124A1349BE
:1057600013481B881288098800880094FFF7E0FD21
:10577000F1E7FFF78DFDEEE7E663FF1F0D64FF1F06
:10578000F241FF1FC063FF1F0E64FF1FA863FF1FCE
:10579000C263FF1FF341FF1FC163FF1FF041FF1FE3
:1057A000AC63FF1FE841FF1FEA41FF1FEC41FF1FF1
:1057B000EE41FF1F10B502A804880B20002C10D169
:1057C000496808784978090201430C48814209D1A7
:1057D000022119800A4B59881170DB7800205BB2D6
:1057E000537010BD074C0A20A142FAD10221198042
:1057F000034B998811705B79F0E7C0466E2A000070
:10580000AC61FF1F6F2A0000F7B5150008AA1688C3
:105810004A680F4F14785278120222430A24BA427F
:1058200014D10122DBB2019200962A0005F024FD7A
:10583000041E0BD1074B1B68002B07D068782A7811
:105840000002104342425041013098472000FEBD03
:10585000022900002064FF1F30B5012503790400F0
:10586000BFB02B4225D01449408805F071F828427A
:105870000CD0124B01A95B8D00220B8002234B80C0
:105880000F4B5B888B80608802F042F90D4960887D
:1058900005F05EF8C0070CD50B4B01A91B88002250
:1058A0000B8002234B80064B9B888B80608802F024
:1058B0002FF93FB030BDC0461864FF1F1C42FF1FC8
:1058C000AC61FF1F1064FF1F7642FF1F10B5074C2D
:1058D0000749200004F0F2FF2000064904F0EEFF23
:1058E0000721054A054804F0ABFF10BDFFFF00008B
:1058F0001864FF1F1064FF1FE0BA00111C42FF1F55
:1059000010B5024802F086FF10BDC046595800117C
:105910000200F0B501270A480A4E51188B1A002BD5
:1059200000DCF0BD0824157843086840384040008A
:10593000805B013C58406D08002CF5D10132EDE749
:10594000FFFF0000FABA0011F0B500250F269D42B6
:1059500000DBF0BD4C5D070944403440A400A05872
:1059600001357840F3E70000F0B589B06A460D00D4
:105970000B000F27110010351C7801332600240975
:105980003E40167054700232AB42F5D12023024AD9
:10599000FFF7DAFF09B0F0BD00BB0011F0B54E789B
:1059A0000B7889B036020C00170001901E43012AC3
:1059B00061D9954B9E4200D877E001339E421CD1BD
:1059C000062A17D1CA788B7812021A430B791B0466
:1059D00013434A7912061A438C4B5A6100221A70FB
:1059E0005A808B4A5A608B4A9A608B4ADA60002050
:1059F00009B0F0BD88225205EEE7884B9E423CD1AB
:105A000082498B78002B00D0F6E00C2A31D10F228E
:105A1000A3789343E27812021343227912041343CA
:105A20006279120613434B60E279A07912020243B5
:105A3000207A00041043627A12060243CA60E27AB6
:105A4000A07A1202024376484A81834208D804238E
:105A50006E49142201980B7005F086FF1420C7E7E9
:105A60001201D21889235B059A42F0D801238B706A
:105A7000BDE7022AFAD00523EAE76A4A01239642E3
:105A8000E6D1FFF705FC052F0CD9E378A2781B02BD
:105A90001343227912041A4363791B061343624AA3
:105AA0000393136005F070FCA1E7584D2B78002B91
:105AB0009DD1AB78002B00D1A0E02B8901339BB2A4
:105AC0000093B34200D091E0132AD4D9CF7C8B7CD1
:105AD0003F02122120001F43FFF71AFF874200D028
:105AE0008EE0002E3DD1E378A2781B021343227989
:105AF000E96812041A4363791B06134303930A22CD
:105B00008B4212D1FF23A370E370237163716B8901
:105B1000002B09D1E37B227C1B0212041343A27BDE
:105B200013431B0901336B8100226B89002B8ED03C
:105B3000002A67D1686837013818000B6B690003C9
:105B40000390984205D9686105F05EFEEB78013359
:105B5000EB7068681022A11C381805F04DFE2E81EC
:105B600045E76F89009A7B1E9BB293423AD1E27857
:105B7000A37812021A43237905A81B041343627900
:105B80006C6812061A43EB6800920392211D0C22E6
:105B9000049305F0E9FE0120260004A940421036D6
:105BA000FFF7E2FE013F012F17D1009A0B23286176
:105BB000824200D04CE704221C49200005F01CFE64
:105BC000042203A9686805F09FFEE968039AFF2391
:105BD000914200D13CE7F73B3AE73100FFF7C4FEC2
:105BE0001036DFE70923B742A4D831E7009BB34260
:105BF00000D9FCE607232BE7022329E7032327E745
:105C0000062325E70A2323E7FFFE00009042FF1F3B
:105C100000000111FFFF00005048593601FF00004D
:105C2000FFFF001102FF000034F000409C42FF1F04
:105C300010B5034C0B000122210000F06BFA10BDDF
:105C4000F15D00110B8870B506000D000224162BC3
:105C500011D92B000322094900F05CFA041E0AD175
:105C6000074B2A881B88191C934200D9111C30004D
:105C700089B200F0EFFA200070BDC0461D5E001131
:105C80003664FF1F10B54A780400013A0B00022069
:105C9000012A07D80A78002A04D0052220000249E8
:105CA00000F038FA10BDC0464B5E00110A7810B5FE
:105CB0000B0004000220002A04D007222000024921
:105CC00000F028FA10BDC046F75E00110A7810B542
:105CD0000B0004000220002A04D0092220000249FF
:105CE00000F018FA10BDC0465D5F001110B5034CFE
:105CF0000B000B22210000F00DFA10BD8D5F00118A
:105D000010B5034C0B000D22210000F003FA10BD6A
:105D1000FF5F001110B5034C0B000F22210000F0B3
:105D2000F9F910BD596000110A7810B50B00040094
:105D30000220002A04D011222000024900F0EAF9D2
:105D400010BDC04669600011002310B51322190070
:105D500000F0E0F910BD000010B5034C0B00172255
:105D6000210000F0D7F910BDBB600011002310B571
:105D70001922190000F0CEF910BD000010B5034C37
:105D80000B001B22210000F0C5F910BDF5600011C9
:105D9000F7B584890D0006000121002C22D00023D4
:105DA0008268D3561778002B1EDA0C2C1AD90C3CBB
:105DB000A4B2131940880093230002F086FE431E0C
:105DC000984101307B06DB0F6B703F23013C1F4085
:105DD000A4B22870AF70AC80002C07D0B368013338
:105DE000AB6000210800FEBD0020EBE7AC60F8E7E7
:105DF0000B7803704B8843704B881B0A83700B79B8
:105E0000C370042070470420022B06D10020537871
:105E100011781B02009A0B43138070470B880370A4
:105E20000B881B0A437002207047042000998342AC
:105E30000AD1537810781B0203430B80D3789078F3
:105E40001B02034300204B807047F8B50D004B78D0
:105E500001240021461C03702B788B4201D82000BE
:105E6000F8BD6B78B01C4F1C012B10D1890069184C
:105E70004B88022233704B88B9001B0A7370691873
:105E800005F03AFC04360434A4B2F9B2E4E7122374
:105E900059436B185A88043132705B8810221B0AF0
:105EA0007370691805F028FC12361234ECE770B5EF
:105EB000049D14001E00052B01D8042070BD6378DA
:105EC00012781B0213432B80E378A2781B02134342
:105ED00002226B802A71211D681D063E05F00CFC14
:105EE000B2B22A81E92AE8D82800A11D0A3005F0BB
:105EF00003FC0020E2E7002310B50A789A4201D89B
:105F0000900010BD9A008A18548801330470548898
:105F1000DBB2240A4470948884709288120AC2709A
:105F20000430EAE710B51100029C062B04D00420CF
:105F30001022142B01D010BD022222714B78087858
:105F40001B0203432380CB7888781B0203436380C2
:105F50000431601D05F0D0FB0020ECE710B50C7893
:105F60008B7804315C43E4B203702200013005F009
:105F7000C3FB601C10BD0420022B06D10020537807
:105F800011781B02009A0B431380704710B50C0068
:105F90000A88023105F0B0FB208810BD70B50400FE
:105FA0000D0004981100012B01D8042070BD167853
:105FB00052781202324302800200F132557014709E
:105FC000E125002C00D10C35023B9AB24280AA4256
:105FD000EBD80231043005F08FFB0020E6E7042007
:105FE000009983420AD1537810781B0203430B8037
:105FF000D37890781B02034300204B80704710B584
:106000000C000A88023105F077FB208810BD0000E3
:1060100070B501211E000420049C0E400B4218D1D3
:10602000CB40DDB28D4214D90A49DBB209889942CE
:106030000FD32300EE331D70330058001118497838
:10604000165C0902314301332152D9B28D42F4D892
:10605000002070BDA842FF1F10B50C000A88023155
:1060600005F04AFB208810BD10B50C788B78043100
:106070005C43E4B203702200013005F03DFB601C7C
:1060800010BD10B511000298032B01D8042010BDDB
:1060900014785278043B120222430280CA788C782A
:1060A0001202224342809AB28280EB2AEED8043157
:1060B000063005F021FB0020E9E710B50C000B8845
:1060C00003700B881B0A43704B8883704B881B0A34
:1060D000C3708A880430063105F00EFBA0880430B6
:1060E00080B210BD0420012B03D100201378009A48
:1060F0001370704710B50C000B8803700B881B0AD7
:1061000043704A880230043105F0F6FA60880230A4
:1061100080B210BDF0B589B003931E4B02924200CD
:106120000700D05A019102F020F81325061E2DD049
:10613000029B01240370019B002B04D000190399DA
:106140009847001984B26B461B7A5BB2002B0FDABA
:106150001021380002F01CFB1925002813D1300053
:106160003219E1B202F066FC051E0CD10C34A4B267
:10617000042304AA380005A993800696948101F0AF
:10618000AFFD051E02D0300005F0CEFA280009B0A0
:10619000F0BDC0463464FF1F70B505000C00002838
:1061A0000CD00020814209D010222000044905F0C3
:1061B000A3FA01202B7823736B78637370BDC046FC
:1061C00040BB0011F0B506000D0017001C0085B0A3
:1061D00002291BD00020102907D1022B07D0102B39
:1061E00003D115E00020102C08D005B0F0BD6946A1
:1061F0003800FFF7D1FF2A0069460BE069463000FE
:10620000FFF7CAFF22006946380004E0022BE9D1FB
:106210002A003900300005F0DFF8E6E7031CF0281B
:1062200000D9F023032008499AB2013A0B80D31712
:10623000034006499B189B100B80D30F04499B1801
:106240005B100B807047C046AC42FF1FAA42FF1F85
:10625000A842FF1F034B1B888B4202D3024B400016
:10626000C1527047AC42FF1F3464FF1F014B400016
:10627000185A70473464FF1F1722014B1A80704769
:106280003464FF1F70B505000E2005F035FB041EB9
:1062900013D0D02303700023062283700749457072
:1062A000033005F029FA064B2100DA8A62811B7E51
:1062B0002373044B187805F0AFF870BD5064FF1FCE
:1062C0004064FF1FFC42FF1F262803D8024B4000FA
:1062D000C05A70470148FCE7AE42FF1FFFFF0000B5
:1062E00070B506000C00094D1C220021280005F0A5
:1062F00053FA074B1E70074B1C7005F0ADFA0123D3
:10630000002801D0002312202B7070BD4064FF1FB5
:10631000FC42FF1F6164FF1F70B505000D4C0800B3
:10632000E260A16010220021656005F045FA0128B5
:1063300003D11021A06802F058FD1022002128008E
:1063400005F03AFA012803D11021606802F04DFDF2
:1063500070BDC0464064FF1F70B5041E05D1002902
:1063600003D006220D4805F0C7F90D4B1D78012D0D
:1063700011D1002C05D102221A7005F03DF9280038
:1063800070BD00221A70074B1B78FF2BF7D020003E
:10639000FFF778FFF3E70025F1E7C0465064FF1FE1
:1063A0004064FF1FFC42FF1F030010B5002801D10D
:1063B000002010BD00780B4A002803D15988D182F3
:1063C0001B7913761378022BF2D10023984200D167
:1063D00003331370044B1B78FF2B01D0FFF752FFE0
:1063E0000120E6E74064FF1FFC42FF1F002911D097
:1063F00000280CD04B79012803D14022524213438C
:1064000003E03F221340032802D001204B71704764
:106410004022F4E70800FAE770B5094D010028783A
:1064200000280BD0074C0622200005F065F921005A
:106430002878FFF7DBFF200005F0A6FA70BDC04604
:106440006064FF1F3A64FF1F00290AD0012808D1A9
:106450003F224B799343C02B03D0403B5A425341D8
:10646000981C704770B5174D06002B78FF2B15D080
:106470000A2005F041FA041E10D0D0230370C83B57
:106480008370114B11491B784670C370062204308B
:1064900005F032F92100287804F0BEFF0C4B1B7880
:1064A000012B0DD10B4B1B68002B03D09B68002BDD
:1064B00000D09847084B04211878084A04F094FF4C
:1064C00070BDC046FC42FF1F6064FF1F3A64FF1F9F
:1064D0005C64FF1F8864FF1F8C64FF1F60EA00007C
:1064E000014B98687047C0464064FF1F014BDB6852
:1064F000186870474064FF1F074B10B5DA681368CF
:1065000001331360054B1878FF2803D08021C9019F
:1065100004F022FF10BDC0464064FF1FFC42FF1F75
:10652000F7B50E0002F0C8F8051E1CD00E4B06622F
:106530001F78002F00D10778AB791020019305F068
:10654000DBF9041E0FD0D0230380C73B8370019B6F
:10655000E91DC3700622043005F0CEF82100380092
:10656000E66004F059FFF7BDFA42FF1F014B1878AF
:106570007047C0466064FF1F054B002805D1054BDE
:106580001A78054B002A00D1014B18007047C0460D
:106590005064FF1F6064FF1F3A64FF1F014B58687F
:1065A0007047C0464064FF1F024B1868431E984165
:1065B000C0B270476464FF1F421E03000120152A09
:1065C00003D9FF3B5A425341D8B27047F0B51C0083
:1065D00000230E0085B0039002920B70029A934242
:1065E00001D3002019E0E55C5A1CD2B2002DF8D08E
:1065F000029851198142F4DC0233DFB2A35C180027
:106600000193FFF7D9FF002807D0013D019A0399B4
:10661000EBB233708A4202D1E01905B0F0BDDB194C
:10662000DBB2DBE710B50C0002F09EF8030012208D
:10663000002B03D02100588805F01EF810BD000083
:1066400070B50E4D84006359002B15D0186A0028D0
:1066500001D005F081F92B59586A002801D005F0C6
:106660007BF92B59986A002801D005F075F9285953
:1066700005F072F900232B5170BDC0467064FF1FF6
:106680001C4B70B504000E00150099420AD11A4B3C
:106690001B68002B01D1122070BD1B68002BFAD0A3
:1066A0009847F9E7154B994215D1134B1B68002BFE
:1066B0000AD01B68002B07D09847002804D1104B44
:1066C0001C70104B1D70E7E729002000FFF7AAFFA0
:1066D0000028E1D1F3E7080001F0EEFF0028DAD04E
:1066E00003780320A342D7D12900300004F0C4FF6F
:1066F000D2E7C046FEFF00006C64FF1FFFFF0000F2
:106700006964FF1F6864FF1FF7B50400808801F00B
:10671000D3FF0025A84203D00578A08802F008F82E
:106720001C4E3378002B1FD0AB421DD11A4B2800D2
:106730001978FFF777FF002818D000233370A3796A
:106740000820A778A688019305F0D6F8011E0DD081
:10675000D0230370CA3B8370019B4770868083718E
:10676000280004F059FE01E0002DE8D1A0880B4B71
:106770008200D358002B01D0FFF762FF1721A088B9
:10678000FFF768FDA08801F027FDA08801F0FEFD5D
:10679000F7BDC0466964FF1F6864FF1F7064FF1F78
:1067A000F0B587B01D000CAB1B88070001930DAB43
:1067B0001B88142002930EAB1B88160003930FABAB
:1067C0001B880091049310AB1B88059305F094F887
:1067D000041E1AD0D0230370CB3B47708370C67061
:1067E000062229000430002D11D004F085FF019B02
:1067F00021006381029B0098A381039BE381049B9A
:106800002382059BA37404F007FE07B0F0BD04F0DB
:10681000C3FFECE7F7B5009308AB1B8807000C201B
:106820000D001600019305F067F8041E13D0280030
:1068300001F042FF00280FD00078D0232370C93B1D
:10684000A370009B21002381019B6770A580E680D7
:10685000638104F0E1FDF7BD014B1878EDE7C04618
:10686000FC42FF1F13B5040064890389C288818834
:10687000C0780094FFF7CEFF13BD000010B5044CA4
:106880002068002803D005F067F80023236010BDBE
:106890007464FF1FA122F0B5818892004A43384BEF
:1068A000384F1B6804009B189D2292009B18827928
:1068B00089B01A603B68002B5FD01D78324B1B6893
:1068C000002B04D05B68002B01D0002098472600E5
:1068D00008363100E079FFF7B7FD237DE071020053
:1068E000E0780493638A29000393238A0293E3895F
:1068F0000193A38800933300FFF752FFE378002B46
:106900000BD1E289A379A18802920196E27928004D
:106910000092012201F0DAFEE0703B68002B20D0EB
:10692000FFF7ACFF194D287800281AD0184B1978BA
:10693000FFF778FE002814D02B78E678082007931C
:10694000A78804F0D9FF011E09D0D0230370CA3BE9
:106950004670837087808671079804F05DFD002380
:106960002B701721A088FFF775FCA08801F034FC7C
:10697000A08801F00BFD09B0F0BD064B9DE7C046B5
:106980003409FF1F7464FF1F8864FF1F6964FF1FC1
:106990006864FF1FFC42FF1FF8B5070008000E00E7
:1069A00001F08AFE041E18D02620FFF78DFC051E7C
:1069B00000D12578062004F09FFF041E0DD0002191
:1069C000062204F0E9FED0232370C23B2100677049
:1069D000A370A680E8B204F01FFDF8BDF0B585B045
:1069E00001930AAB1B78070002930BAB1B780800DE
:1069F0000D000092039301F05FFE061E22D01020CE
:106A000004F07AFF041E1DD01022002104F0C4FE01
:106A10002620FFF759FC002800D13078D0232370BE
:106A2000C13BA370009B21002372019B67706372BE
:106A3000029BA580A372039BC0B2E3720C9BE36030
:106A400004F0EAFC05B0F0BDF7B50D00019001F0CF
:106A500033FE071E20D00E2004F04EFF041E1BD074
:106A60002620FFF731FC061E00D13E78D02323807C
:106A7000C53B0622A370F91DE01C04F03DFE019BFE
:106A80002A0063810123DD401A401D40210022734A
:106A90006573F0B204F0C0FCF7BD0000F0B585B03E
:106AA000029010000D0017000A9E039301F004FEEF
:106AB000041E31D0029B002B2ED1039B02795B0771
:106AC00024D5122313430422002E08D10B99002948
:106AD00005D10C99002902D10D9900291AD01A4329
:106AE0000D9B2271002B00D0C9E0002E00D1CFE019
:106AF000002D00D0CCE0606A002801D004F02CFF0B
:106B00001C21300004F0E8FE606205E002239A4395
:106B10000E33D7E793432371654BBA00D458002C4A
:106B200000D1AAE0002E10D0236A002B03D11C2034
:106B300004F0DAFC20625E4BBA00D358186A0028D1
:106B400003D01C22310004F0D7FD0C9B002B12D087
:106B5000574CBB001D596B6A002B03D1162004F063
:106B6000C3FC6862BB00E358586A002803D01622B1
:106B70000C9904F0C1FD0D9B002B11D04C4DBC00B5
:106B80006659B36A002B03D1142004F0ADFCB06247
:106B90002B59986A002803D014220D9904F0ACFDFB
:106BA000380001F089FD051E67D0414BBA00D3586B
:106BB000002B62D01A6A3420002A00D11C389A6A4D
:106BC000002A01D0143080B20B9A002A01D01C3068
:106BD00080B25B6A002B01D0163080B204F08CFECC
:106BE000041E4AD01822002104F0D6FD2620FFF70B
:106BF0006BFB0190002801D12B780193D0232370E7
:106C0000029B200063700A23294EA370039BBD00E2
:106C1000A371AB59A780196A1830002905D01C222E
:106C2000A06004F069FD200034307359996A00298E
:106C300007D0030014221433E060029304F05CFDDB
:106C400002980B9B002B08D003001C221C330B99CD
:106C50002061029304F050FD02987359596A00298B
:106C600003D01622606104F047FD6B4621001879BD
:106C700004F0D2FB3800FFF7E3FC05B0F0BD1022B2
:106C80000D9B0D991B69A018236204F035FD2CE7BC
:106C90000B9B002B00D13FE7012D00D03CE7606A41
:106CA000002801D004F058FE1C210B982AE7C046AA
:106CB0007064FF1F10B5044C2068002803D004F056
:106CC0004BFE0023236010BD6464FF1F0B4B07B510
:106CD0001A68002A01D100200EBD6946531C01200C
:106CE00012780731FFF772FC0028F4D002780123F4
:106CF000100018401A42EED0EEE7C0468064FF1F35
:106D0000F0B51F4F01203B6887B0002B25D09B7842
:106D1000059300F0B3FB002821D00A20FFF7D4FA36
:106D200004000B20FFF7D0FA164B05001E78731EE7
:106D30009E413B68F6B2191DD878FFF757FB3B68B8
:106D40002900DA7A043303929A790193029200902F
:106D500033002000059A04F0EFFB07B0F0BDFFF709
:106D6000B5FF002805D00620FFF7AEFA0400072083
:106D7000D8E70820FFF7A8FA04000920D2E7C046A8
:106D80006464FF1F6064FF1F70B50A4E040033780F
:106D90000D00FF2B0DD0042004F0AEFD011E08D025
:106DA000D0230370CE3B45708370C470307804F0FC
:106DB00033FB70BD0C43FF1F70B5040006200D00AF
:106DC00004F09AFD011E0AD0D0230370CD3B8370DE
:106DD000054B44701B688580187804F01DFB002C5F
:106DE00001D0FFF767FF70BD6464FF1FF8B5264F41
:106DF00006003B680D001124002B05D10522234B12
:106E00001B78134202D112242000F8BD204A10241E
:106E10001268002AF8D01278002AF5D0DB0719D5BD
:106E20002B789A1E012A1AD80C2004F05DFB13243B
:106E300038600028E8D000230A2243702900067039
:106E4000023004F059FCFFF75BFF041E0AD0FFF785
:106E500031FFD9E700F012FB0028E1D1E4E7002B75
:106E6000E2D0D0E70B4B1B78032BCDD11D20FFF7D1
:106E70002BFA094B18800028C6D0084B042118783B
:106E8000074A04F0B1FABFE76464FF1F6164FF1FA3
:106E90008064FF1F6064FF1F5E64FF1F8C64FF1F20
:106EA00060EA0000F7B50193194B14001A78052326
:106EB00006000F0012201A4221D0012920D1154BC3
:106EC0001D68002D1BD002201F2C18D8002C02D0CA
:106ED000019B002B13D0104B1F221E706E1C002133
:106EE000300004F059FC01992200300004F004FC49
:106EF000310020002C70002F06D004F015FDFEBDDF
:106F0000064B12201D68DCE704F016FCF7E7C046CC
:106F10006164FF1F8064FF1F0C43FF1F7C64FF1F21
:106F2000F8B50F4E12243368002B17D01B780F3C96
:106F3000834213D100250B4F0221387804F07CFBEB
:106F4000094B042138781D8004F076FB074B28009C
:106F50001D8033685C7004F007FA04002000F8BD5F
:106F60006464FF1F8C64FF1F7864FF1F5E64FF1F53
:106F700070B5012823D11B4C2388002B03D01A4A5B
:106F80001578002D07D0194B1B68002B02D01878FC
:106F9000FFF7C6FF70BD3B2B02D93C3B2380F9E7CE
:106FA000134E0221307804F047FBFA222388920026
:106FB00002215A43307804F0CFFA2580EAE70B4BE0
:106FC0001B68002BE6D00B4B1B785B07E2D5084B08
:106FD0000221187804F030FB0022024B1A80FFF7E0
:106FE00069FED7E77864FF1F5C64FF1F6464FF1FBE
:106FF0008C64FF1F6164FF1FF8B51E4D28680028D0
:1070000003D004F0A9FC00232B601B4E306800283D
:1070100003D004F0A1FC00233360184F05243B7813
:1070200018002040234221D0154800F02BFA3B786D
:10703000234213D0202004F057FA2860002813D0F0
:107040002022002104F0A8FB202004F04DFA041EA9
:10705000306005D02022002104F09EFB002004E0D7
:10706000286804F079FC2C601320F8BD00F00AFABF
:10707000F4E7C0468064FF1F7C64FF1F6164FF1F4C
:107080000043FF1F10B50A4C23681A1E0ED00028BB
:1070900008D10130587004F067F9002805D0236842
:1070A000002B02D00021FFF787FE0122100010BD47
:1070B0006464FF1FF7B5274E050033680191181E61
:1070C00021D05C78244F012C30D1FFF7FFFD002840
:1070D00025D02000FFF7F8F80400412814D91F4BF1
:1070E000022118781E4A04F07FF91E4B3C3C1C809C
:1070F000022233685A703B78002B14D12800019982
:10710000FFF75AFE0120FEBDFA2292004243002AF8
:10711000EED0124B0221187804F01EFAE8E7FFF7D0
:10712000D3F80200F3E700233B70EBE73B78002B3A
:10713000E8D1032004F0E0FB011E08D0D023037047
:10714000CC3B457083703368187804F065F9FFF71D
:10715000B1FDD7E76464FF1F5C64FF1F8C64FF1FF1
:1071600060EA00007864FF1F10B5174983880200A9
:107170008B4220D011D815498B4217D014490020DA
:107180005B1899B2012907D8926811785A42534185
:10719000D8B2FFF7F9FD012010BD0E4A00209B1860
:1071A00007229BB29A424041C0B2F5E78368187843
:1071B000FFF768FFF0E7836899785A780902187832
:1071C0001143FFF777FFE7E70A20000006200000E1
:1071D000F8DFFFFFAFDFFFFF014B18707047C046BD
:1071E0000D43FF1F10B5064C207001F041FA2078C6
:1071F00004F092F90521207800F062FD10BDC04630
:107200008C64FF1F0BB273B50D00002B00DBC4E0D4
:10721000884B187804F0B0FB041E0ED00378912B35
:107220000FD0A22B00D1A1E0834B1878FF2852D0B9
:10723000210004F0F1F800284DD1802000026840C0
:1072400076BD43780F2B76D013D8052B70D00E2B3C
:10725000EAD18088794B98422BD8794B98421BD839
:10726000784B9842E0D1A3681878591CFFF774F85E
:1072700038E03E2BD8D18378032B74D06CD8012B07
:107280006ED0022BD0D1704B1B68002B23D05B68D3
:10729000002B20D098471EE06C4BC0180C28C3D898
:1072A00004F012FB1DC2C2150BC20B0B0B3223C222
:1072B0003C00674BC0180728B6D8664B1B68002BEC
:1072C00009D01B68002B06D0200098470AE0A3686D
:1072D0001878FFF7C7F8200004F01EFAADE7A068A1
:1072E000FFF762F800289FD0F5E7A3681B78002B12
:1072F000F1D0554B1B68002BEDD01B68002BEAD05A
:10730000210055489847EDE74F4B1B68002BE2D012
:107310001B68002BDFD021005048F3E7504B1B685F
:10732000002BD8D05B68002BD5D021004348E9E77B
:10733000FFF7EAF9CFE780884A4B984203D04A4BDF
:10734000984200D070E7464B1B68002BC3D05B68A7
:10735000002BC0D02100D5E7153B012BBBD963E73B
:10736000FFF798FAB7E7FFF77DFAB4E73F4B1B78D2
:10737000042B07D100236A4613800179408800F06E
:10738000C5FCA8E7364B1B68002BA4D05B68002B1C
:10739000A1D00100364898479DE7012421420AD038
:1073A000294B1B68002B04D05B68002B01D0002008
:1073B0009847012043E78B070AD5264B1B68002B13
:1073C00004D05B68002B01D020009847022036E7EC
:1073D0000421280008400D4200D131E7254E3388B2
:1073E000002B21D0013B9BB23380002B1AD1FFF739
:1073F000DBF800280AD0204B1C70164B1B68002BB2
:1074000004D05B68002B01D020009847FFF7C6F836
:10741000694601F001FD6846FEF7FEFF1D20FEF7FC
:1074200053FF308004200AE7024B187804F004F977
:10743000F8E7C0468C64FF1F0D43FF1F0E200000BD
:1074400001200000091000008464FF1FFEDFFFFF21
:10745000AFDFFFFF8864FF1F0C2000000B2000003F
:107460006C64FF1F0D200000132000006164FF1FEB
:10747000FFFF00005E64FF1F5C64FF1F10B501F09A
:107480009BF910BD014B18607047C0468864FF1F10
:107490000B880020162B01D817230420014A1380E3
:1074A0007047C0463664FF1F00207047074A03003C
:1074B0001188814207D091880020994202D1013081
:1074C0008000101870470020FAE7C0469464FF1F40
:1074D000F0B58F7806000D00C5B01E2F15D1FFF74F
:1074E000E5FF051E03D10024200045B0F0BD0022B9
:1074F0003B003100C078009200F0B2FB0400A81CF1
:1075000000F0D2FBFF23EB70EEE7264B062403933B
:107510001B78FF2BE8D0182FE6D87B08224A013BC6
:10752000DB0002929A589446002ADDD0029AD318C2
:107530005B68002BD8D00878002802D14B78012B4B
:1075400002D10624122FCFD107AFAB8869780097FC
:107550006446AA68A047041EC6D1AB78029A5B08AD
:10756000013BDB00D318390030005B689847041EEC
:107570000BD1AB78042BB6D0039A310010782200DF
:10758000009700F06DFB0400AEE76A78002AABD1EB
:10759000AA7805A93B88087130000A704B80FEF775
:1075A00047FBA0E71043FF1F50BB00111D4B37B531
:1075B000050098420BD000290AD1FFF777FF002879
:1075C00005D11948FFF772FF002800D0058037BDAC
:1075D00001291AD1FFF76AFF041EF8D001235B428C
:1075E0000380A378FF2BF2D0FE2B07D00023E07896
:1075F0001422009329001E3300F032FBA01C00F07F
:1076000053FB01235B426380E1E70229DFD10139AB
:1076100001F0BEF80028DAD12800FFF747FF041E6A
:10762000DFD1D4E7FEFF0000FFFF0000022210B50B
:10763000074B52421A80074801325A809A80DA80FA
:1076400000F07EFA044801F025F8002010BDC04685
:107650009464FF1FD1740011AD7500110388F7B554
:107660000400002B02D102252800FEBD4268022141
:10767000137825485268FEF7A5FD00282ED0234F29
:1076800001253A88002AEFD0802321885B0201255A
:107690009B1A9942E8DC0C2003F026FF061E31D02D
:1076A0003B8822889C4600231800019561469DB2C4
:1076B000491989B2AA421BD8002801D062443A80F5
:1076C00000233000082208C0210004F015F8104AF9
:1076D0001368002B13D100251660C5E762680221EC
:1076E00013780C485268FEF76DFD0028C7D1BAE741
:1076F00060681D014019418101330198D6E71A00E5
:107700001B68E6E71325AFE7BEBB00110E43FF1F62
:107710009064FF1FBCBB0011014B18707047C0463E
:107720001043FF1F14230A0010B51A40194204D059
:107730000122102101F048F810BD4B06F9D40120B8
:1077400088434000F8E710B514008B0604D50122E9
:10775000102101F039F810BD08230A001A4019421F
:1077600002D14BB2002B0FDA102101F02DF80028C6
:1077700008D02300F2331B78002BECD0F1342378AF
:10778000012BE8D10020E6E703208907FAD4E2E7DD
:10779000F0B51F00184B85B01C6801900291039250
:1077A000002C27D1200005B0F0BDA5683301ED18ED
:1077B0006B89019A934211D3029A93420ED8002FFB
:1077C00004D10A9B002B10D12C00EBE73B00297859
:1077D000039A6868FEF7F6FC0028F2D10136B6B2CB
:1077E000A388B342E1D82468DAE7A3680A9A5B89E0
:1077F0001380E9E70026F3E79064FF1F37B50C001C
:107800000A8849880123914217D3002A15D0651DA3
:1078100023792A0002210A48FEF7D4FC102300280D
:107820000BD023796188208800242A000094FFF778
:10783000AFFF0A23A04200D0230018003EBDC0467F
:10784000BEBB001113B50A0008884988012388428D
:107850000BD8002809D00024137905320094FFF7D3
:1078600097FF0A23A04200D02300180016BD13B5CD
:107870000A0008884988012388420BD8002809D0CB
:107880000024137905320094FFF782FF0A23A042F7
:1078900000D02300180016BDF0B58BB003904A88C5
:1078A00008880E000123824255D3002853D00023BC
:1078B000012704AC23700022718813000092FFF7A7
:1078C00067FF051E3ED02078002835D12B78022B8B
:1078D00018D167706A8983000130E31880005A80EC
:1078E00069680222201803F007FF23780133DBB216
:1078F0002370042B19D93B006889013080B2002B1A
:10790000D9D01FE002236370122358436A892318D9
:1079100004305A8069681022201803F0EDFE2378A5
:107920000133DBB22370002BE5D10C4A6B899B1825
:107930005A425341DBB2DFE76378012BE4D12B7865
:10794000022BC7D022780A23002A04D021000398F2
:10795000FEF798F9002318000BB0F0BD0100FFFFFF
:107960000F4BF0B504001868002816D083685D89B5
:10797000A54207D88288AE18B44203DA12019A18D9
:10798000934201D10068EFE71E005F891036A742DD
:1079900004D1002900D00D801800F0BD3300EFE7BE
:1079A0009064FF1F70B505000C0008880021FFF7E8
:1079B000D7FF03000120002B04D022002800197AF1
:1079C000FFF7C1FE70BDF7B50C0000250190230044
:1079D000EE331B78AB4201D800200AE06B00E65A78
:1079E00000213000E718FFF7BBFF002802D12680F6
:1079F0000130FEBD017A0198FFF794FE002802D005
:107A00003B882380F5E70135EDB2E0E710B50400CF
:107A100008880021FFF7A4FF03000120002B03D0FA
:107A20002000197AFFF77EFE10BD0000054B1B6891
:107A3000002B01D1180004E09A6852898242F6D1E5
:107A4000988870479064FF1FF0B50E27002687B016
:107A5000039302ABFF183E8005001F4B40891400C2
:107A6000984207D02B78013000976A6880B2FFF700
:107A70008FFE060002212B7818486A68FEF7A2FBE9
:107A800000280FD06C892000FFF7D0FF002802D01B
:107A9000013C0419A4B2039B002B00D01C803000D1
:107AA00007B0F0BD02212B780D486A68FEF78AFB0B
:107AB0000028E7D102212B780A486A68FEF782FB8A
:107AC000002807D0002EDED03B88A342DBD174898A
:107AD000013CDFE76C89DEE7FFFF0000BEBB001161
:107AE000BCBB0011BABB001110B50C00FFF7DEFCE7
:107AF00003000220002B0AD0002C00D023609B78CA
:107B00001720FE2B03D00138FF2B00D1002010BD21
:107B100073B50D0001A904001600FFF7E5FF172853
:107B200005D0002E04D129002000FEF727F976BDEC
:107B300001221021200000F047FE0028F3D0F6E7D4
:107B4000014B18607047C046A064FF1F37B56B46F5
:107B50009D1D010004000222280003F005FF2B8870
:107B6000B02B0ED12379122B09D12300FA331B78C5
:107B7000012B06D10121608800F0E0F801E01B2B09
:107B8000F8D037BD10B5054B0421187000F098F8F7
:107B9000FFF74CFDFEF770FB10BDC046A464FF1F4D
:107BA0000020F0B50BB20F0087B0834234DA274BC8
:107BB000187803F0E1FE051E2BD00378A02B25D109
:107BC00003AE3100FEF7E4F8041E0BD1B378DB07F7
:107BD00024D51F4B06341B68002B03D03100688866
:107BE00098470400A868002801D003F09DFD002CF0
:107BF00008D1184A039B1340174A934206D0B37822
:107C00001B2B03D00121688800F098F8280003F0AE
:107C100083FD80200002784007B0F0BD0F4B1B6849
:107C2000002B10D0310068889847041EDAD0737892
:107C3000002BD7D1B27801A90A704B800C716888EB
:107C4000FDF7F6FFCEE70624F1E7C046A464FF1F68
:107C50009C64FF1F00FFFF0000011200A064FF1FD3
:107C6000F7B50190FC200D0017001E0003F044FE44
:107C700004001320002C12D0B02320002370089B96
:107C8000F4226770658026710830002B08D0190037
:107C900003F032FD2100019803F0BEFB0020FEBD81
:107CA000089903F079FDF5E710B5041E06D00078B9
:107CB000FD2803D803F088FCFF23237010BD0000CB
:107CC0000A1F93B210B504000220032B05D882408E
:107CD0000020024BD1529B189C7010BDC464FF1F42
:107CE0000B8870B5043B04000D000220032B0BD859
:107CF0000121200000F04CFD03001420002B03D0D4
:107D00002900200000F0DEFB70BD000007B5130065
:107D1000034A00920A00012100F02CFC0EBDC0466F
:107D2000497F001107B5019203220092024B0A001D
:107D3000122100F049FC0EBDC77F001107B56B464C
:107D400001AA11800449D88008780633012802D19D
:107D5000190003F041FD07BDA564FF1F0C4B10B5D2
:107D600018700023FF210B4A1380138193819380A5
:107D7000094A53801370517293819372D174D382E4
:107D80001375517703F010FB00F0FCF910BDC046ED
:107D9000D464FF1FC464FF1FA664FF1FF0B58DB03D
:107DA0006B46002003910C229B5E834200DBB0E017
:107DB0005D4B187803F0E0FD051E00D1A4E00378C8
:107DC000902B00D09DE006AF01004688380000F0FF
:107DD00013FA79680400002900D19CE03B88052B48
:107DE0006ED13B89032B1CD905AC200000F0A2F812
:107DF0006288172A61D83989131D994231D179686F
:107E0000237804310291D90738D5607800F08EF9D3
:107E1000071E06D0002303712378012B08D0132BF3
:107E200023D0A868002800D178E003F07DFC75E03D
:107E30006288029909A800F0A6F80290380000F0C4
:107E40008BF909AA2378387A019200223100009236
:107E5000029A00F012F9380000F064F9029B002B3E
:107E6000DFD0300000F080F9DBE70378032BD8D1B6
:107E70006288029909A800F0D6F8DEE7122B13D128
:107E8000029909A800F0B5F8021EEAD127498B88AB
:107E9000002BC6D0887909A92378019161780091D7
:107EA000310000F0EAF8BCE7002302AA9383300017
:107EB000617809AAFFF72AFFB3E71D4B0993F6E79C
:107EC000042B02D09A1F012AABD8184A043B9B000E
:107ED000995A0029A5D0D218907831003A0000F0C4
:107EE000AEF800289DD13B88042B03D0012130003F
:107EF000FFF724FF012C04D1A868002801D003F06B
:107F000013FC280003F008FC8020039B0002434080
:107F100018000DB0F0BD012800D182E7012130002A
:107F2000FFF70CFFEDE7C046D464FF1FC464FF1FDA
:107F3000010017000B7803704B784370CB788A7878
:107F40001B021343438070470A88030002700A88AB
:107F5000120A42700A88012A06D14A8882704A8829
:107F6000120AC2700420704702208242FBD14A8864
:107F700004309A704A88120ADA708A881A718A88DC
:107F8000120A5A71EFE710B50400012082420CD9A1
:107F90004B780A781B0213432380834206D1CB78A7
:107FA0008A781B0213436380002010BD022BFBD193
:107FB000CB788A781B02134363804B790A791B02C2
:107FC0001343A380F0E70B8803700B881B0A4370F0
:107FD0004B8883704B881B0AC3708B8803718B8816
:107FE0001B0A4371CB888371CB881B0AC37108209D
:107FF000704703000120082A14D14A780878120239
:1080000002431A80CA788878120202435A804A7959
:108010000879120202439A80CA79887912020243CF
:108020000020DA80704710B504000120022A05D133
:1080300000204B780A781B021343238010BDF8B54B
:10804000060010200F00150003F056FC040001206C
:10805000002C0ED0A0230C22290023806780201D35
:10806000002D07D003F048FB2100300003F0D4F9C5
:108070000020F8BD03F090FBF6E7F7B51E00009076
:1080800008AB142017001D78019103F035FC041E85
:1080900012D0A2230370019B47704380099B057196
:1080A00046710C220830002B07D0190003F024FB86
:1080B0002100009803F0B0F9F7BD099903F06CFBBB
:1080C000F6E737B5041E0FD04388002B0CD00025EF
:1080D000C1881323007A172201950095FFF7CDFF81
:1080E000FF2365806372257037BD000010B50C4911
:1080F00004004A88002A09D08B89002B05D0002073
:10810000CB8A0222834201D010BD012213000A2033
:10811000434300204032C854C81842800472F3E739
:10812000A664FF1F0023438003707047094B0021A2
:108130001A0010B55C88002C06D01C79844203D14B
:108140000A234B43D01810BD01310A330329F1D162
:108150000020F8E7A664FF1F10B50400407A03F082
:1081600033FAFF23637210BD7047043010B580B23C
:1081700003F06AF9002803D00421494203F004FA0D
:1081800010BD000070B50025104CA0682580A581A9
:10819000A580A84202D003F0C7FAA56000250C4CC8
:1081A0000C4B606D1D80230058331D70A84202D017
:1081B00003F0BAFA656500256068002801D003F075
:1081C000B3FA013508340A2DF6D170BD6C65FF1F76
:1081D0001065FF1F6065FF1F70B5041E09D1054DB6
:1081E0002880A881A880A868002802D003F09CFA03
:1081F000AC6070BD6C65FF1FF0B54B8885B0019316
:10820000002343600A7905000F00022A00D07BE0BA
:10821000CA88032A17D98B685E7819783602DC7809
:10822000D8790E4399781B7A24021B020C4303432E
:1082300053495BBA0B80331D93421ED1042C04D0EA
:10824000631F022B0ED9012015E0019A4D4B12013C
:10825000D35A002B06D00198FFF7BEFF4A4A136994
:10826000013313610421B8682E812C80494203F048
:108270008BF96860002005B0F0BD434D042C06D09A
:10828000631F022B0FD9EB680133EB60DBE7019A28
:108290003C4B1201D35A002B05D00198FFF79CFFED
:1082A0002B6901332B61374B30000293019B029AFB
:1082B0001B010193002301998C468B5213006344E8
:1082C0009C8003939E81FFF750FF039B041E9860E0
:1082D00016D00421B868494203F056F9FA88010023
:1082E000043A200003F008FA0199029AFB888A5A9E
:1082F000043B9B18029A8B522B6801332B60A2E738
:10830000AB690133AB619EE71E4B0293019B1E01DB
:10831000029BF35A002B2DD002998C19A0680028DB
:1083200028D0012A26D1FA889B189BB27352A189C2
:10833000994217D39B1AC018B96803F0DDF9029B64
:10834000A289F35A934200D07DE700222B81A388B3
:108350002B80A3686B60029BF2520B4A5368013377
:10836000536070E7084A9368013393600198FFF700
:1083700033FF68E7044A536901335361F6E7C046A7
:10838000D664FF1F6C65FF1FDC64FF1F70B5051E00
:1083900015D10B4C0B4B1880230058331870606DAF
:1083A000002802D003F0C0F96565250050356068EB
:1083B000002801D003F0B8F90834AC42F7D170BD01
:1083C0001065FF1F6065FF1FF0B51700A12285B083
:1083D000920001934243394B06001B680C009B1826
:1083E000D933FF331D78FDF741FF0430854204DDAA
:1083F0003000FDF73BFF0430C5B2BD4207D33A0061
:1084000000213000019B03F09FF905B0F0BD290069
:10841000380003F049FA2300C6B250331E700393AC
:10842000019B29006365380003F0F6F9CBB2029393
:10843000002B02D0039B01361E7000262300503310
:1084400003931B78B34204D8606D002831D100201B
:10845000DBE7029A2800002A04D0013B1000B34257
:1084600000D02800F700E719387003F06DFA786043
:1084700000280ED03A78019903F03EF9019A3B7832
:108480000136D3180E4A0193D369F6B20133D36192
:10849000D4E7039B18706065A74205D1084A1320F2
:1084A000D36A0133D362B0E7606803F03DF9083462
:1084B000F2E703F039F900236365C8E73409FF1FC9
:1084C000DC64FF1FF7B50D0007000421686803F0A6
:1084D0005BF82B89040003702B891B0A43702B88DF
:1084E00083702B881B0AC3702E8902250436F6B2CE
:1084F000F42E15D81B4B9F4214D10C2003F0FCF92D
:108500001135011E0CD0902303708E3B0371043B88
:108510004380154B8460C680187802F07DFF0025EB
:108520002800FEBD5C237B43104AD31800935833C8
:1085300001931B78002B0FD1030032003800009903
:10854000FFF742FF019B05001B78002BE8D13800A4
:10855000009903F0C9F8E3E7054A0725536A013398
:108560005362DDE7FEFF0000D464FF1F1065FF1FAC
:10857000DC64FF1FF0B587B0009017200F001600D5
:108580000193FFF7F2FD1325041E19D00C98031E6A
:1085900002D00199201D9847030AE370052302AA1F
:1085A000A0700430908127700098667003A99380B2
:1085B0000494FFF787FF051E02D0200003F0B4F8F3
:1085C000280007B0F0BD0000F0B587B01F000CAB6D
:1085D0001B780391059301210DAB06001C780492D2
:1085E00000F0D6F81425002821D02000FFF77EFDEA
:1085F0000135041E1BD01149059B0A780370013216
:10860000D2B2131EC68001D101231A000B70227151
:108610003000049B03990097FFF7ACFF051E09D1BA
:10862000230021000648074A093302F035FF2800DD
:1086300007B0F0BD002363802370F8E7D864FF1F04
:10864000C380001130750000F8B505000E00064C1F
:10865000064F2368002B02D03100280098470434CD
:10866000BC42F6D1F8BDC0467C65FF1F9065FF1F78
:108670000123064A5B425380002313715362044A6C
:10868000136053609360D360136170479065FF1F60
:108690007C65FF1F0200002310B506499C000859A5
:1086A000002801D1625010BD0133052BF6D11320F3
:1086B000F9E7C0467C65FF1F034A5388181A4342F6
:1086C00058414042104070479065FF1FF0B585B09B
:1086D00002930AAB1F780CAB1B88009008000E00B9
:1086E00001920393FFF7E8FF05001120002D1BD135
:1086F0000E48FFF7E1FF04001520002C14D00622DD
:108700000B99A771E01D02F0F7FF019B3000237168
:10871000029B29006371009B66802370039B656246
:10872000E381FFF791FF280005B0F0BDFFFF0000D7
:1087300010B5FFF7C1FF04000220002C12D06088A2
:108740000121FFF781FF606A002801D003F004F9DE
:1087500028220021200003F01FF8012300205B42A3
:108760006380207110BD000030B5074A074C558862
:10877000010013780020A54204D05B1A59424B41F6
:108780005842104030BDC0469065FF1FFFFF0000FB
:10879000084A10B501230C00904208D0FFF78CFF67
:1087A000031E04D0037923405A1E9341DBB2180004
:1087B00010BDC046FEFF0000024B1879431E9841D1
:1087C000C0B270479065FF1F70B504000D00160021
:1087D000FFF772FF002804D10D4B9C4200D01430EB
:1087E00070BD416A03790520002907D012221A4082
:1087F000102A02D10520002EF2D10F20DB06EFD582
:10880000897E0C20A9428941494249420840E7E754
:10881000FEFF0000030010B5002800D110BD034882
:10882000034A41889142F9D09847F7E79065FF1FC6
:10883000FFFF0000002330B5C45CCD5C6C40D45415
:108840000133102BF8D130BD0F23002210B5C45CCA
:1088500064002243CA54C25CD209013BF7D210BD66
:108860000200010010B52032103102F045FE10BDAB
:10887000F0B58BB00390102005931700049102F01F
:1088800033FE0090102002F02FFE009B1324019075
:10889000002B05D000280CD11324009803F05CF8BD
:1088A000019B002B02D0180003F056F820000BB0FB
:1088B000F0BD102002F018FE0600102002F014FE99
:1088C00013240500002E00D1AEE0002819D010229C
:1088D000002102F061FF32002900039802F00CFE33
:1088E000041E0ED133787F2B51D830000099FFF74A
:1088F000ABFF009B1B787F2B53D801990098FFF7A3
:10890000A3FF300003F028F8002D02D0280003F068
:1089100023F8002CC1D1102002F0E6FD0600102043
:1089200002F0E2FD0290002E7CD0002878D03A00C0
:108930000F3223000125121105D00F333B4015B231
:108940005A4253411BB26A1E1201002B33D0049BC2
:10895000D2B298180099029AFFF76CFF013D1022DD
:108960000021300002F018FFADB2049F2D017D19E7
:10897000AF4242D0002C33D0300002F0EDFF029B1A
:10898000002B00D189E7180002F0E6FF85E72900F7
:108990003000FFF759FF28002549009AFFF74AFFEA
:1089A000A7E729000098FFF74FFF28002049019A08
:1089B000FFF740FFA5E70F210F4004998A18D9B2AD
:1089C0008F4208D9D15C06A819540133102BF6D177
:1089D000029A0199C0E7791A48424141C901F2E778
:1089E0003900300006AAFFF725FF3200039806A9D8
:1089F00002F082FD10370400BAE7002CBCD1300031
:108A0000029906AAFFF716FF320006A9039802F0A2
:108A100073FD082204003100059802F06DFEABE7FB
:108A20001324A9E71324AAE7002800D06EE733E750
:108A3000C4BB0011F0B58BB00F00160002250090EA
:108A400000283FD0002A3DD00B1DDBB21800029356
:108A500002F04AFD1135041E34D0FDF747FD050034
:108A60003A000099201D02F01FFDEBB20393E37062
:108A70002B0CDBB22F0A00936370FFB22B0E237016
:108A8000A7700193FDF72CFD1022010006A802F04B
:108A90000BFD2100029A04AB06A8FFF7E9FE051EB4
:108AA0000DD1039B08223370009B04A9B370019B76
:108AB0007770F370301D02F0F7FCFDF71DFD20000C
:108AC00002F04AFF28000BB0F0BDF0B58FB00D00EA
:108AD000149E039004920593002A03D102242000DF
:108AE0000FB0F0BD002EF9D00398FFF7E5FD142478
:108AF000071EF4D07278337812021A43B3781B043D
:108B00001343F27812061A43036A0192934201D387
:108B10000133E3D1002D03D03B7901249B07DED53F
:108B20000822002106A802F037FE059B1324043317
:108B3000DBB21800029302F0D7FC051ECFD0059AD5
:108B40000499043002F0B0FC04223100280002F045
:108B5000ABFC3900102210310AA802F0A5FC290054
:108B6000029A06AB0AA8FFF783FE041E0FD1082263
:108B700006A908A802F098FC0822311D08A802F0F6
:108B80002BFC012807D101990398FDF7C9FC2800A7
:108B900002F0E2FEA3E70124F9E7000070B51C4CE7
:108BA00005002368181E10D0002D14D11A78002A51
:108BB0000CD1981C083202F09FFD02F0FDFB01353C
:108BC000002808D123681D70012070BD0A331800E9
:108BD000082202F091FD2368002BF5D0122002F04C
:108BE0008BFE061E0DD0C123216803704570023133
:108BF0001022023002F080FD23683100587802F024
:108C00000BFC206802F0A8FE00232360DCE7C046CE
:108C1000B865FF1FF8B504002020FDF755FB0D4E89
:108C2000A700BB590500002B0DD000280BD0D87829
:108C3000FF2809D108492A000C55F3590748033386
:108C4000611802F029FCF8BD290002F01DFC002883
:108C5000F0D1F8E7D465FF1FBC65FF1F6D9E0011C2
:108C600070B5064D84006359002B05D0D87802F00A
:108C7000ABFCFF226359DA7070BDC046D465FF1F9C
:108C800070B506008CB00C0015000021302268463B
:108C900002F082FD31001022684602F005FC1D2022
:108CA00021000322684402F0FFFB6846FFF7D8FD6D
:108CB0002D21040003222800694402F0F5FB200066
:108CC0000CB070BDF0B50700160097B001931CAB57
:108CD0001D7830221EAB00910AA800211C7802F0FA
:108CE0005BFD102239000AA802F0DEFB10220021F1
:108CF00002A802F051FD0722310002A802F0D4FBC5
:108D0000072202AB9818631E9C41019902F0CCFB2C
:108D100002AB9C732B005A1E934102AAD37300210D
:108D2000102206A802F038FD06221D9907A802F0BD
:108D3000BBFB1A2002ABC01806221F9902F0B4FB3D
:108D4000102200990EA802F0AFFB102202AB0EA970
:108D500008781C78013A6040D2B2087001330131C2
:108D6000002AF5D10AA8FFF77BFD102212A9040002
:108D70000EA802F0C1FC102206AB0EA908781D78DF
:108D8000013A6840D2B2087001330131002AF5D1AE
:108D90000AA8FFF765FD044310222098E4B212A947
:108DA00002F082FB200017B0F0BD70B50E00140079
:108DB0008CB00100102268461D0002F075FB3100E6
:108DC000082204A802F070FB2100082206A802F085
:108DD0006BFB6846FFF744FD04001022280008A939
:108DE00002F062FB20000CB070BDF8B506000D006B
:108DF00000243719AC4200D3F8BD02F00DFC030A81
:108E00003B70631CDBB201379D4203D90234F0543E
:108E1000E4B2EEE71C00EDE773B506000C00022596
:108E2000002819D0002917D0032101A8FFF7DDFF82
:108E30006B469A793F231A40013313436A46300048
:108E4000937101A92200FFF71BFF051E04D1032225
:108E5000E01C01A902F050FC280076BD03785807F9
:108E6000DA08C00FD20080009B0710439B0F184305
:108E7000C0B2704707230B40C908C9000B430370F9
:108E80007047000070B50400FFF7EAFE134DA40020
:108E90006359002B21D0186A002801D002F05CFD34
:108EA0002B59986E002801D002F056FD2B59D86E30
:108EB000002801D002F050FD2B59186F002801D076
:108EC00002F04AFD2B59586F002801D002F044FDF2
:108ED000285902F041FD00232B5170BDD465FF1FBE
:108EE0000E4B8000C35870B50C00002B0FD09D684E
:108EF000002D0CD02B78201D0B706B784B70A97C4B
:108F0000FFF7B8FF2B7E23726B69E36070BD102200
:108F10000021200002F040FCF8E7C046D465FF1FA6
:108F2000014B18607047C046D065FF1F074A030019
:108F30008000825810B5002A06D0D088984203D10C
:108F4000012901D1FFF79EFF10BDC046D465FF1F68
:108F5000F0B5264E95B087000B93BB5905000991DB
:108F600012200A92002B31D0D888FFF7A5FB04000D
:108F70001420002C2AD0280010A9FFF7B1FFBB59FC
:108F80001E781D6A002E23D00895FDF7EFFA070022
:108F90000020FDF7F1FA0790A379E61D069310ADC6
:108FA0000CA9089800F0E2FA0EA9280000F0D7FA00
:108FB0000B9B0A990493069B09980293079B0396BF
:108FC000019300970EAB0CAAFFF77CFE15B0F0BD25
:108FD000FDF7CCFA06903000FDF7CEFAE31DA77935
:108FE000079310AB06000893DAE7C046D465FF1F6D
:108FF00030B50C4C85002A59030085B00120002AA9
:109000000ED018006946FFF76BFF2B591A78D888E5
:10901000054B002A00D1054B6A46072100F0D9FB19
:1090200005B030BDD465FF1F5F9500116D9500112F
:1090300030B5094C8500295985B010226846253184
:1090400002F05AFB2A591121044BD0886A4600F0DD
:10905000C0FB05B030BDC046D465FF1F09960011A6
:1090600030B5094C8500295985B010226846353144
:1090700002F042FB2A591121044BD0886A4600F0C5
:10908000A8FB05B030BDC046D465FF1F4796001150
:10909000F7B54D4F86001020F4590D0002F024FA68
:1090A000F3592062186A132200286CD0033A290071
:1090B0009C6802F021FBF3591A780192002A58D1DA
:1090C0001E6A227D317B944651400122019F11424C
:1090D00001D167461740217D914339432175377B84
:1090E0004F40BC4660460027800701D44F08174018
:1090F000012102208F40227D82433A432275377B33
:109100005740BC4660460027400701D497080F40EF
:109110000420227DBF0082433A432275627D0027EE
:1091200094466046727B42400A4201D167460F4036
:109130000121627D8A433A436275777B5740BC4682
:1091400060460027800701D457080F400220627D47
:109150007F00824317436775767B00227E40760747
:1091600001D4BA080A400426617D9200B1430A4343
:1091700062756A78002A08D06278002A05D0052234
:109180000533DA7700221000FEBD0422297911424E
:1091900005D1A17C114202D10533033AF1E7019ACE
:1091A00021782C78002A02D10A002100140018220C
:1091B0000429E8D8042CE6D805206043034A053387
:1091C0001218525CDDE7C046D465FF1FD4BB001106
:1091D00010B50A001121024B00F0FBFA10BDC04689
:1091E000A39600110B0030B587B001AD2B806B4604
:1091F00004001100981D082202F07EFA2A000B21BB
:109200002000024B00F0E5FA07B030BDCB9600110C
:1092100010B50A001121024B00F0DBFA10BDC04668
:109220001F97001113B50B0011006A4613706B46AF
:1092300004000622581C02F05FFA6A46082120004A
:10924000014B00F0C6FA13BD3F97001110B50A009C
:109250001121024B00F0BDFA10BDC0468F970011DE
:109260007FB505000B4BAA00D4580800002C0FD086
:10927000666F237FE28821780396266F0296E66E5A
:109280000196A46E0094FDF709FC2800FFF7FAFD93
:109290007FBDC046D465FF1F10B51721FFF7E0FF63
:1092A00010BD000070B50A000D00064B022104003D
:1092B00000F08FFA060029782000FFF7D1FF300078
:1092C00070BDC0466F96001170B586B000236A4627
:1092D0001370836804001D78681E0A2859D801A9F4
:1092E00002F0A2FA060633373B3F43474B4F530089
:1092F000180000F042F9062312284BD000281BD199
:109300006088FFF7D9F90823002813D04279002A92
:1093100047D1264B1A78072312070BD5244B1A681E
:109320000723002A06D01668002E03D0290001AAC0
:10933000B04703006A4613706B461B786088002BA9
:109340002AD1FFF767FC06B070BD180000F06CF979
:10935000D4E7180000F087F9D0E7180000F093F97F
:10936000CCE7180000F0ADF9C8E7180000F0C3F929
:10937000C4E7180000F0F6F9C0E7180000F0F6F9AD
:10938000BCE7180000F013FAB8E7180000F013FA71
:10939000B4E707236A46137069466088FFF782FFC7
:1093A000D1E70523012AC5D1024BB8E76164FF1F4D
:1093B000CC65FF1FD065FF1FF8B52C4F8600F35911
:1093C00004000D00002B40D0DA8882423DD15A784B
:1093D000062A33D11A78002A2ED0012099681A6AF9
:1093E000097D014206D0157B054203D007225A7041
:1093F0000120F8BD0220014204D0157B054201D0B6
:109400000922F4E70420014204D0127B024201D079
:109410000B22ECE7164B1B68002BE9D05B68002B96
:10942000E6D020009847BB5900215B78122BDFD192
:109430002000FFF715FFDBE70E4BECE7112A04D104
:10944000002900D032252900F2E7002D08D12000A4
:10945000FFF732F9002803D0102302791343037178
:1094600021002800FDF798FAC2E7C046D465FF1F27
:10947000CC65FF1FD065FF1F70B50E4E8500AB5940
:109480000400002B13D01B78002B11D10A4B1B6852
:10949000002B04D05B68002B01D020009847735943
:1094A0005B78122B03D100212000FFF7D9FE70BD9D
:1094B000024BECE7D465FF1FD065FF1FCC65FF1F93
:1094C000094B8000C3581020002B0CD01A6A002AC8
:1094D00009D09B68002B06D0127A1B7E101C9A4282
:1094E00000D9181CC0B27047D465FF1F70B50300C7
:1094F0000D0014000220002A30D000292ED0137055
:109500000B78081D53704B789370FFF7A7FCE07041
:10951000012002212B7A23716B7B034063716A7BEC
:109520000A401343042263716E7B16403343637118
:109530006E7BF608F600334363712B7B0340A37107
:10954000287B014000200B43A371297B0A40134371
:10955000A3712A7BD208D2001343A37170BD10B54A
:109560000A0001000120FFF7C1FF10BD10B50A007D
:1095700001000220FFF7BAFF10BD70B506000C0015
:109580000220002E30D000292ED07378201D0B70C1
:10959000B3784B70F178FFF76DFC012235792572B5
:1095A00071794B100800134093401040034388101A
:1095B00010408000C9080343C9000B436373B179AD
:1095C0004B100800134093401040034388100240A2
:1095D0009200C9081343C9000B4321202373FCF7F1
:1095E00073FE854201D2122070BD2220257AFCF73D
:1095F0006BFE8542F7D823781820042BF4D86378C3
:10960000012BF1D80020EFE7030010B5022000295C
:1096100009D0002B07D00322481C0A7019000D3214
:1096200002F06AF8002010BD03000222080010B505
:10963000002B06D0002904D00E32591C02F05CF831
:109640000022100010BD030010B50220002909D02F
:10965000002B07D00422481C0A7019000C3202F0BB
:109660004BF8002010BD10B5FFF7DEFF10BD030062
:109670000220002906D0002B04D0052200200A7009
:109680001B784B70704703000220002B08D0002984
:1096900006D05B7800200B70013B082B00D91830F6
:1096A0007047030010B50220002909D0002B07D015
:1096B0000622481C0A7019000A3202F01DF8002028
:1096C00010BD10B5FFF7B0FF10BD02000B00022067
:1096D00010B500290ED0002A0CD00721197011886E
:1096E00059701188090A997011180822D81C02F0C3
:1096F00003F8002010BD03000A00022010B5002B63
:109700000CD000290AD099785878090201431180B9
:10971000901CD91C082201F0EFFF002010BD0300AF
:1097200010B50220002909D0002B07D00822481CC0
:109730000A701900921801F0DFFF002010BD02002E
:109740000B00022010B500290BD0002A09D00921F6
:109750001970117818185970511C062201F0CCFFAD
:10976000002010BD10B5FFF75FFF10BD02000B0019
:10977000022010B5002A09D0002907D051781970AD
:1097800011180622581C01F0B7FF002010BD03007D
:1097900010B50220002909D0002B07D00A22481C4E
:1097A0000A701900063201F0A7FF002010BD10B5A5
:1097B000FFF73AFF10BD02000B00022010B5002A8F
:1097C00006D0002904D018005178FFF753FB002081
:1097D00010BDF0B585B017001E006A4606230500CF
:1097E000080091819380FEF7C0FC1324011E0290B3
:1097F0000CD03800B047041E05D1280001A9FEF79F
:109800006FFA041E02D0029801F08EFF2800FFF7C5
:1098100001FA200005B0F0BDF0B504008BB0019155
:1098200015000021102202A801F0B6FF334EA70058
:10983000B85900283CD0C388A34239D10378002B03
:1098400036D14278062A18D102000100553235314E
:109850000C3006ABFFF7A9FA002829D12000FFF74A
:109860002FFE020006A902A801F046FF200002A96F
:1098700001F05AFE01200BB0F0BD816E002917D017
:109880000B8A112A28D19D420ED101981231093A32
:1098900001F0A2FD012807D1BB5920009D6EFFF702
:1098A0000FFE29000200DEE732212000FFF7D8FC7E
:1098B0002000FEF701FF061E1BD0416A002918D0C8
:1098C0000B8AAB4215D108220198123101F084FDB8
:1098D00001280ED1716A0AE09D42E9D1082201985F
:1098E000123101F079FD0128E2D1BB59996E8A7ECF
:1098F000B9E7200001F0B0FDBCE7C046D465FF1F0A
:10990000F0B56B4D87007E5985B033780290039394
:10991000002B00D087E0B368346A01937078062882
:1099200017D101221B7D134202D0217B114218D195
:109930000222134202D0217B114251D10422134250
:1099400003D0237B134200D08BE0019B5A7DEB595F
:1099500091E007380428F8D801F066FF032E42672B
:109960008300B36E002B03D11C2001F0BDFDB06657
:10997000EB599C6E002C1CD010220021200001F01D
:109980000BFF0298FFF79CFD01002000FFF72DFA66
:1099900001F042FE2082200008211230FFF725FA54
:1099A0000298FFF78DFDA076EB592100D888FFF7CC
:1099B0000FFC0822EB591CE0B36E002B05D01A00F7
:1099C000198AF0881232FFF70DFC0222019B197DE3
:1099D000EB5911423DD0207B10423AD0073208E0CB
:1099E000F488FCF7DBFD01002000FFF711FC0A22E0
:1099F000EB595A70029B9C002A595378073B042B61
:109A000011D8D088FEF758FE00284ED0C3895A08D6
:109A1000D2182849029B0298CB542B594118043381
:109A2000254801F039FD05B0F0BDFCF79FFD0300AE
:109A30000120834201D100200393EB59DE88FCF71B
:109A40009BFD039902003000FFF7ECFB019AEB59F4
:109A5000117D042211420CD0217B114209D00B222E
:109A6000C7E7F688FCF73CFD01003000FFF7EEFB8E
:109A70006BE7019A527D01210A4204D0607B0842C3
:109A800001D00C22B5E702210A4204D0607B0842D3
:109A900001D00E22ADE704210A4204D0627B0A42C3
:109AA00001D01022A5E71222A3E7FA225200B0E764
:109AB000D465FF1FD865FF1F779E001110B5064BB8
:109AC0001A780423100018401A4200D00348FFF708
:109AD00027FA002010BDC0466164FF1F1443FF1F1A
:109AE00070B50400FFF7D4FA051E43D12000FFF73C
:109AF0007FFA234EA400A0598268937CDB0708D527
:109B00000321036A1B790B40012B02D1017F0B4318
:109B10000377431DD97F8B1E022B0DD8022900D05D
:109B20000121C088FCF790FF042133591A7F597036
:109B30000A431A77280070BD01290CD10223102294
:109B4000437000210C3001F027FE305910213530D0
:109B5000FFF74BF9EEE70529ECD10223D11843704A
:109B600010220C3001F0C8FD04233259117F0B4341
:109B70001377EAE708251828DCD1053DDAE7C04667
:109B8000D465FF1FF0B58BB0059143887E4F9E00D2
:109B9000F45915000493002C15D1012902D000209E
:109BA0000BB0F0BD101D57781678FFF757F9EB682A
:109BB000320002932B7A0499019300903B0020001D
:109BC000FCF70CFFEBE7E388049A934201D00820EE
:109BD000E6E72378012B00D1D4E0059B581E092825
:109BE00000D9CFE001F020FE05CE0A29CC506C85CB
:109BF0009AB229000498FFF773FFD1E720002900EB
:109C00001022453001F078FDB9594B78042B02D170
:109C1000013B4B70C3E70B000A00253335320C3192
:109C20000498FFF795F90498FFF702FA0522431EFE
:109C30009841BB59C0005A70B2E720002900102299
:109C4000553001F059FD049B4F4C9D002959049853
:109C50000A0006AB55320C31FFF77AF92959102268
:109C6000453106A801F0B8FB012808D10498FFF798
:109C7000F7F90590002804D106222B595A7005984F
:109C80008EE708230593FAE763780C2B7AD1E36E0D
:109C9000002B03D11C2001F027FCE066BB59D86ED5
:109CA00000286FD01022290001F026FDBB5904982E
:109CB000DC6EFFF705FC0D22A076BB595A706EE7EB
:109CC000E06E00285ED063780D2B5BD12B880822D4
:109CD0000382A91C123001F00FFDBB599A68517D17
:109CE0000222114226D0186A407B104222D00C3248
:109CF000E4E763780E2B45D1236F002B03D11620A8
:109D000001F0F2FB2067BB59186F002803D0102226
:109D1000290001F0F1FC0F22BB59CFE763780F2B2C
:109D200030D1206F0622691C103001F0E5FCBB59D0
:109D30009A68517D0422114203D0196A497B11426D
:109D4000D5D100210498FFF78BFA28E7636F002B29
:109D50000DD0BB59586F0028F3D01022290001F014
:109D6000CBFC0122BB5952425B6F1A61E9E7142018
:109D700001F0BAFBBB5960675B6F002BE9D126E7A6
:109D80002978DFE707200BE7D465FF1F10B5064CE5
:109D9000207001F069FC06212078FDF791FF03484F
:109DA000FEF778FC10BDC046E765FF1F2D8F001140
:109DB00000200BB270B50D00834216DA264B1878DE
:109DC00001F0DAFD041E0DD00378922B0ED0A02BEB
:109DD00037D0224B1878FF283AD0210001F01CFB25
:109DE000002835D180200002684070BD43780E2BDA
:109DF0000BD03E2BEDD18378052B12D0082BE8D168
:109E000081798088FFF7D8FA08E0154B82889A425A
:109E1000DFD183681878591CFEF7C0FE002817D1DF
:109E2000D7E7104B1B785B0712D50F4B1B68002B35
:109E30000ED09B68002B0BD0C289811D808898476B
:109E4000ECE7FFF741FAA068002801D001F06CFCB4
:109E5000200001F061FCC5E7E765FF1F0D43FF1F10
:109E6000182000006164FF1FD065FF1F10B5007847
:109E7000FFF712FA10BD10B50078FFF7FDFA10BD1C
:109E80000C234343084A10B59B185A68002A03D094
:109E9000012901D1904710BD9B68002BFBD0002900
:109EA000F9D19847F7E7C0460466FF1F01238340B6
:109EB000094A10B5946B1C439463506B98435063EC
:109EC000D46B20009843012901D120001843D063AE
:109ED000116B0B43136310BD00800040F0B50024EC
:109EE0000127154B85B0DA6B144E03921A6C019260
:109EF000DA64019BE3403B4217D0039DE5403D40BF
:109F00000295E5B202992800FFF7BAFF316A736A39
:109F1000002908D03900002B01D00299794028008F
:109F2000FFF7C4FF01E0002BF9D101340C36172CE8
:109F3000DFD105B0F0BDC04600800040E865FF1FDE
:109F4000064B01215A68C2400A4204D01B68C34034
:109F50001800084070471B6DF9E7C04600800040BC
:109F60000122064B8240002903D0D9680A43DA60F7
:109F70007047D9689143D960FAE7C046003800407D
:109F800030B5032444430F4BE25C1B199C785D7889
:109F900001232D1B0135AB40013BA340A140DB4316
:109FA0000C00122807D8084992005218116819406D
:109FB0002143116030BD054A11680B4023431360F3
:109FC000F8E7C0461BBC001108F0004014F0004048
:109FD000C21F70B5D4B20623092C0BD80125084C3A
:109FE0009540002908D00021FFF7CAFF23682B43C2
:109FF00023600023180070BD2368AB43F8E7C04618
:10A0000000380040214BF0B51B185B78022B21D1A2
:10A01000032444431E4A1F4EA35C12199478012264
:10A0200015008540B76B013CE4B23D43A240B563E7
:10A03000194C122815D89B0000290CD117495B1820
:10A0400099680A439A600123205C154A834011688D
:10A050000B431360F0BD11495B18996891439960F7
:10A06000F1E70E4B00290DD159690A435A61225C70
:10A070001328E8D00123203A93400A490868034393
:10A080000B60E7E7596991435961F0E7E865FF1F05
:10A090001BBC00110080004060BC001100F00040BB
:10A0A000A0F00040A4F00040F8B500241B4E1C4D69
:10A0B0001C4B1B5D012B1FD1194A9269E2401A42C9
:10A0C0000BD00122B25693402200143AD2B2022A97
:10A0D00009D815494A6913434B61013402360C35DE
:10A0E000172CE5D1F8BD0022B2560F499200521844
:10A0F00091680B439360F0E7022BEED1E7B2380092
:10A10000FFF71EFF01235840C1B23800FFF77AFF66
:10A110003800FFF715FF6877DFE7C046EDBB001199
:10A12000E865FF1FE965FF1F00F0004001220238CB
:10A130008240054B002903D059690A435A61704790
:10A14000596991435961FAE700380040F8B50E00AB
:10A1500001210F008740114A0400D368FD43BB432F
:10A16000D360831E8B4201D8FFF7E0FF002120005F
:10A17000FFF72EFF0A4A0B4B5168012E05D13943D8
:10A180001B1951605E700020F8BD29405160022209
:10A190001C1962709A6915409D61F4E7003800400F
:10A1A00000800040E865FF1F012210B58240074B88
:10A1B000002906D019680A431A600121FFF7C6FF7B
:10A1C00010BD196891431960F7E7C0460080004050
:10A1D0000C2370B5002543430A4A29009B181D70C3
:10A1E000094B04001B185D70FFF7B0FF0123A3406B
:10A1F000064928000A681A430A6005490A689A4312
:10A200000A6070BD0466FF1FE865FF1F34800040D0
:10A210003080004070B504000E00FF2813D00325E5
:10A220000540FFF7D5FF084AA3089B009B183F2273
:10A23000ED00AA40AE4019682000914331431960F7
:10A240000121FFF78DFE70BD18380040F8B50C24D1
:10A250004443134B0500E4186368002B03D1A36843
:10A260001220002B1AD0022201270E4B00215B196D
:10A270005A7028002770FFF769FF63681E1E08D018
:10A28000A3683E00002B04D02800FFF759FE46408B
:10A29000F6B228003100FFF709FE0020F8BDC046E5
:10A2A0000466FF1FE865FF1FF7B5C420FF222B4B94
:10A2B00080001958002491433F3A0A431A508022E3
:10A2C000274F5202274E1A60274B1D5D002D21D0CB
:10A2D000A31E012B03D80121E0B2FFF727FF012DB8
:10A2E00018D11F4B9B69E3402B4213D0E3B21800F7
:10A2F0000193FFF725FE01000198FFF755FFE3B238
:10A30000143B022B1DD801217156184A8D40536908
:10A31000AB4353613B7F002B0DD0E5B22800FFF724
:10A3200095FF2800FFF70CFE7B7F0100834202D0DF
:10A330002800FFF7A5FD01340C370236172CC3D1D6
:10A34000F7BD012100237156F3568D40074A9B004B
:10A350009B189A68AA439A60DCE7C04600E100E0D7
:10A36000E865FF1FEDBB0011E965FF1F00F000402D
:10A3700010B501210400FFF7E9FE0123044A002083
:10A3800011194B70A34091690B43936110BDC046F6
:10A39000E865FF1F70B50E0015000400FFF718FFF9
:10A3A0000C236343094A20009B189D605E60FFF701
:10A3B0004DFFF021064B074A8900051E5A5002D076
:10A3C0002000FFF705FF280070BDC0460466FF1F90
:10A3D0000000FF1FDD9E001170B5134D07202C7883
:10A3E000002C1FD1982221005200280000F0ECFF21
:10A3F0000123C420FF222B700C4B80001C635C6384
:10A400000B4B1C605C600B4B195891433F3A0A435D
:10A410001A50802252021A600D20074A074901F0A3
:10A420004BF8200070BDC046E865FF1F008000406B
:10A43000A0F0004000E100E0A9A20011A9A00011D5
:10A44000030010B50620072B09D8054A137000F049
:10A45000D3FFD7210020034B034A89005A5010BD77
:10A460003C43FF1F0000FF1F8D1BFF1F70B51D0029
:10A4700002240C2910D8094ACA40D2070CD5FBF790
:10A480002FFF041E08D1059A04992800FBF744FF0A
:10A49000FCF7B2FDFFF712FB200070BD12100000A8
:10A4A00030B50D7802232C009C43184201D02B4379
:10A4B0001C0008252300AB43284201D02B00234376
:10A4C00020241D00A543204201D01C4325002A233F
:10A4D0000D70184204D011781E3B0B43137030BD31
:10A4E0000028FCD10C2113788B43F7E7F8B51D0049
:10A4F00006AB1B88140007AA0E000B201778002B50
:10A5000027D10A78022A49D14A6850781178000286
:10A51000244A08438018042840D801F085F9031222
:10A520001D1B2300F06801F08FF8021CC0B2B84276
:10A5300000D93A1CD2B22000F1682A8001F0DCF880
:10A5400006E00222F3681B882A8023701B0A6370CE
:10A550000020F8BD0622EEE701232B80F3681B786C
:10A560002370F5E7F368002B16D008222A801A889A
:10A5700022701A88120A62705A88A2705A88120AC7
:10A58000E2709A8822719A88120A6271DA88A2713E
:10A59000DB881B0AE371DBE72B80D9E701202B80E6
:10A5A000D7E7C04600D6FFFFF7B516000A781D00B2
:10A5B00008AB1F880C000123022A18D14A68507882
:10A5C000117800022B4A0843801803280FD801F0A5
:10A5D0002BF902254439E06801F036F8C0B20723B0
:10A5E000B84204D37B190193152B02DD0D2318000B
:10A5F000FEBDE0682A003100C01901F07DF86B460D
:10A6000000209B88E268D0541B4B1B68834203D018
:10A610001B68834200D098470023E8E70B23002FF4
:10A62000E5D1022DE2D1737832781B021343E26840
:10A630001380114B1B68002BEED01B68002BEBD056
:10A640000120E8E70B23002FD1D1062DCED12A001F
:10A650003100E06801F050F8DEE70B23002FC6D18F
:10A66000012DC3D132787533012AC0D8E3681A703E
:10A67000D2E7C04600D6FFFFF467FF1F70B50C009D
:10A680001500072837D801F0CFF8041436361B36EA
:10A69000242E182015290BD8184E16220021300020
:10A6A00001F07AF822002900300001F025F800209E
:10A6B00070BD18200229FBD11288114B1A80F6E7D1
:10A6C00018200829F4D10A000E48290001F04CF99D
:10A6D000EDE718200129EBD10B4B10780B49DA6913
:10A6E000FFF7DEFEE3E718200129E1D1064B1078E1
:10A6F0000749DA6BF4E70220DAE7C046DC67FF1FA0
:10A70000BA43FF1FB043FF1F4043FF1F6843FF1FB3
:10A710008843FF1F030010B50020DB0704D5072185
:10A72000024A034800F08CF810BDC04678BC001106
:10A730004043FF1F054A03001068002803D08288A9
:10A740009A4201D1806870470068F6E7EC69FF1F04
:10A750000A88030008009A4204D08A8804309A428A
:10A7600000D0002070470000F8B5F22200230D4F02
:10A770000D4E7968050042433370994200D07B60EA
:10A780000A4C0021200001F007F800231A007C6029
:10A79000AB4202D100203370F8BD01332280DBB21E
:10A7A000F234F5E7E46AFF1FE26AFF1FF069FF1F5A
:10A7B00073B56B4601900600684615001980FCF7DA
:10A7C0004DFF041E11D1002D0FD07689002E11D01F
:10A7D0000C2000F089FE00280ED0084A046013689F
:10A7E00086808560002B02D11060200076BD1A00A3
:10A7F0001B68F7E70224F8E71324F6E7EC69FF1F6C
:10A80000012100220A4B10B549420A4C1980998057
:10A810009A719A70084B2070012019805A60FFF7D6
:10A82000A3FF2078FCF778FF0448FDF733FF10BD45
:10A83000FC67FF1FEC6AFF1FE46AFF1FEDA8001111
:10A84000022310B5002802D0FFF7B2FF0300180062
:10A8500010BD0000030010B50020DB0704D5042163
:10A86000024A0348FFF7A4FF10BDC0468CBC00118C
:10A87000C043FF1FF0B50E2687B003930CAB1F88B3
:10A8800002ABF6180500080031000292FDF768F8E7
:10A8900004000120002C0FD03088FFF74BFF03008D
:10A8A0000E20002B08D05E68002E05D02100280065
:10A8B000039B029A0097B04707B0F0BD0A4B10B552
:10A8C000984207D10122002352420A808B708A806D
:10A8D0008B7110BDFFF73CFF0028FAD001235B42CB
:10A8E000038000238370F4E7FFFF0000F8B5050044
:10A8F00001290AD1134E00243388F227AB4219D024
:10A9000028001149FFF7DAFF06E0022904D10139D6
:10A91000FDF73EFF0028EDD0F8BD3B0063437268B1
:10A92000D018D35A002B09D03A00002100F034FF90
:10A930000134E4B2054B1B78A342EED801235B42FD
:10A940003380DDE7E46AFF1FFC67FF1FE26AFF1F39
:10A9500010B5FFF7FDFE03000020834200D0987879
:10A9600010BD0000F0B589B01C000EAB80CB039089
:10A970001E8810AB1B78049202930B7A0D00DB0645
:10A9800016D42B780593022B24D00498FFF7D2FE1F
:10A99000002812D003689C46002B0ED0029B220098
:10A9A000019329003B00644603980096A04705E008
:10A9B0000498FFF7BFFE002802D10E2009B0F0BDB9
:10A9C0008368002BF9D00A222900039898470028B1
:10A9D000D7D0F3E76B6858781A786B4B00021043B6
:10A9E0009842D2D8043B984210D2684B984242D049
:10A9F00015D8674BC0180128C7D80B20002EDDD111
:10AA0000EB681A7859683A80200028E0614BC0183A
:10AA1000032800D979E000F007FF846A789E5E4B36
:10AA20009842B2D10B20002EC8D101233B80EB68A5
:10AA300031001B7823706889013080B2FCF790FFE9
:10AA40003A88031E0ED0017802328A183A80428971
:10AA500062704289120AA27059680278E01C00F004
:10AA60004BFE06E004323A8031000422601C00F004
:10AA700093FE0020A2E70B20002E9FD1EB6807A9D0
:10AA80001E8804233B80330A300026706370FCF775
:10AA900067FF051E28D004AB9A890E2304A95B1812
:10AAA0003E49C668FCF7D0FF00280BD12B783C4804
:10AAB0006A680599FBF786FB002803D1012304AAE5
:10AAC0005B42D3813278022A06D17168201D00F0E2
:10AAD00013FE3B8802333B800E2304AA9B181B887D
:10AAE000A3701B0AE370C4E704ABDE81F4E70B201C
:10AAF000002E00D062E7E9680398FFF729FF0223E0
:10AB00003B802070000A6070B3E70B20002E00D05D
:10AB100054E70222EB681B883A8023701B0A63709B
:10AB2000A7E7E86800F090FDC2B203000720B24238
:10AB300000D243E70DD00299DBB27118994202DBD3
:10AB4000921BD3B20293029BE9681A003B808919D9
:10AB50005AE70023F6E70B20002E00D02EE707224D
:10AB6000EB683A801A7822705A7862705A88A2701C
:10AB70005A88120AE2701A792271DA886271DB88C7
:10AB80001B0AA37175E7C0460429000002280000D3
:10AB900000D8FFFFFFD6FFFF03280000FFFF0000E3
:10ABA000BCBB0011F0B58DB06B460020089120228F
:10ABB0009B5E83423DDAA64B187800F0DDFE071E4F
:10ABC00032D00378B02B2CD10079023816281FD848
:10ABD00000F04AFE17001E001E001E0031001E007D
:10ABE00096001E001D011E0052011E0073011E0072
:10ABF000CD011E0050021E001E001E008E021E000F
:10AC0000E302944B94491B8878880B80FBF71AF871
:10AC10003800FCF79BFF914B1B68002B01D03800DC
:10AC20009847380000F078FD8020089B00024340E0
:10AC300018000DB0F0BDEE220021874800F0ACFDF9
:10AC40000BAA3B7B7989388900923A000D32FCF7D8
:10AC50009FFD0400804B1B78002C3FD146E0804BC9
:10AC6000788805937F4B4100CB5A0BAE073BDBB294
:10AC700032880293002301937B4B210006930093BB
:10AC8000059BFFF76FFE744D002810D1069B3A8A92
:10AC90001B889A420BD138000599123000F09CFBBA
:10ACA000002804D02B7862899B00EB185A80162369
:10ACB00006A81B18328820007989FCF7C5FE2B787E
:10ACC00004009A00AA1851880029C3D00133DBB2CE
:10ACD0002B70002807D006A9C98A9180634A128880
:10ACE0009A42BCD802E0012149429180002B04D055
:10ACF00059497888FAF7DAFF8AE73E890A2479E029
:10AD000000253E89574B06937B88069A5B009B5A29
:10AD1000033B9D4202DB002DF0D05BE0162206A82B
:10AD200012183B7B798900923A0030000D32FCF713
:10AD30002FFD0590002858D04689017A7888FCF7C5
:10AD4000F1FC041E44D1464B78880793069B4100D2
:10AD5000C95A454B0439C9B206AAD28A0693029150
:10AD6000019400930599079BFFF7FCFD041E2FD16A
:10AD7000069B39491A88931C002D26D14B8079886F
:10AD8000384B4900CB5A5119033B8B4220DD059BC0
:10AD900031485B8941190B71A91C0135C9B2EDB26B
:10ADA000059145191B0A2B71059B2D490433181871
:10ADB00000F0A2FC2C4B059A1B88D318DDB22C4B5B
:10ADC0009E4205D00136B6B29CE749889942D6D05A
:10ADD000002D0CD0204C2800618800F025FB20704D
:10ADE00021007888FAF772FF12E7059CF0E7002C43
:10ADF00000D183E77B78142B00D109E716493B7912
:10AE00004E800B700C717888FAF712FF00E7162459
:10AE100006ABE41821003889FCF7A2FD011E00D121
:10AE2000B7E1788822880F4C45002C5B0A4D013C25
:10AE3000E4B2029400240F4B01940095FFF792FDB9
:10AE4000041E00D014E129007888FAF74FFFDFE6EE
:10AE5000EC6AFF1FAC42FF1F0468FF1FF867FF1F6B
:10AE6000F868FF1F3464FF1FE869FF1FAA42FF1F35
:10AE7000FFFF00000668FF1F162406ABE418210040
:10AE80003889FCF76DFD011E00D182E178882288A7
:10AE9000AE4C45002C5BAE4D013CE4B202947C8983
:10AEA000AC4B01940095FFF75DFD041E00D0DFE080
:10AEB00029007888FAF724FFAAE60025A44B1D8014
:10AEC0003B00F6331B78A24A78880792AB4208D938
:10AED0009E4B12880693069943005B5A013B9A42A7
:10AEE00003DB0799FAF716FF92E616246B00FB18AE
:10AEF000059306ABE418059B21001889FCF730FD8B
:10AF0000011E03D1059B01241E8973E77888924BAB
:10AF10002288069C099343001B5B904E013BDBB2E9
:10AF20000293002300960193099BFFF71BFD041E6B
:10AF300002D0059B1E895DE77B88069A5B009B5AC1
:10AF4000079A108832881218934202DC1B1A013BC0
:10AF500033807F4C023032880999001900F0CCFB15
:10AF60002388328801359B182380EDB2A8E70BAA0D
:10AF70003B7B7989388900923A000D32FCF708FC56
:10AF800000250590059B002B04D10A24002D00D13B
:10AF90006EE060E0059B7888197AFCF7C3FB01003E
:10AFA000041E63D1694C6C4B788806940993069B08
:10AFB0004400E45A694B063CE4B20BAE3288079376
:10AFC0000294019100930599099BFFF7CBFC041EA5
:10AFD0004CD1079B5E491B881A1D002D30D14A8039
:10AFE000059B5B4C5A8963191A716B1C9BB2E31861
:10AFF000120A1A71162306A832881B187989059837
:10B00000FCF722FDFF21AA1C2E1D03350B00059025
:10B0100092B2B6B2ADB2002803D006ABDB8AD9B289
:10B020001B0AA218651911712B714C4D301D2A880D
:10B030004949201800F060FB2B88F618B5B2A1E74B
:10B040004988914207D17A8806995200525AEB18E2
:10B05000053A9A42C4DC3E4C2800618800F024FC8A
:10B06000207021007888FAF75FFED1E5002DF2D13B
:10B070003E89BFE6162606ABF61831003889FCF784
:10B080006FFC3D000400FA3500282DD0037A9B06A2
:10B090000CD400227B893989788800923A000C32DE
:10B0A000FFF7E8FB041E10D03E8915E03088FFF75B
:10B0B00041FB00281AD08368002B17D021001222F0
:10B0C00078889847041EE4D0EEE72B78002B02D155
:10B0D0007888FAF739FE00262B78002B00D097E508
:10B0E000002C00D194E585E60124DDE70E24DBE7A2
:10B0F000162506ABED1829003889FCF731FC041E33
:10B1000047D0037A9B0611D4154A7B88118899424F
:10B1100003D01448814207D11380134BF2261D78C7
:10B120000023D9B2A94221D30924A1E72888FFF737
:10B1300001FB00282FD08368002B2CD02100122285
:10B1400078889847041EDFD092E7C0463464FF1F1A
:10B150000468FF1F0668FF1FF868FF1FE869FF1FEC
:10B16000E46AFF1FFFFF0000E26AFF1F310059433E
:10B17000546801336018615A0029D2D13C00083468
:10B180002100F22200F0B8FA21007888FAF7E4FDF5
:10B190003EE501246CE70E246AE71D4B1A887B8884
:10B1A0009A4231D07888FAF7E1FD31E5F22305982B
:10B1B00051684343CD18C95A00291FD03B7A012B4F
:10B1C0000BD16C88AB887888AA1D0094FFF752FBDE
:10B1D000041E02D000233B722E88F2220021280098
:10B1E00000F0DAFA00232B80059B0133DBB20593D4
:10B1F000084B05991B78064A8B42D7D801235B423E
:10B200001380002CCED0F5E5002634000596EFE73C
:10B21000E46AFF1FE26AFF1F70B504000E0015000C
:10B22000FFF796FA031E08D131000548FFF790FAA0
:10B2300003001120002B02D01C8000209D7070BDE7
:10B24000FFFF0000F8B50B4F06003B780D0014001F
:10B25000FF2B0ED00A2000F04FFB011E09D0B123B6
:10B260000380002346800371C5800481387800F094
:10B27000D3F8F8BD0144FF1FF7B50F0008A9060079
:10B28000088809A90B240988002821D10234022B3F
:10B290001ED1557813782D021D432B008B4301934B
:10B2A0007334002B14D1FB68300019000093FFF7B2
:10B2B0004FFB019C85420BD02A0030000099FFF71C
:10B2C000ABFF041E04D12A0030007989FFF7BAFFD2
:10B2D0002000FEBDF0B50E7885B003900AA8058861
:10B2E0000120022E0DD14C682778647824023C435B
:10B2F000054FBC4205D10398DBB201960095FFF7DC
:10B30000BBFF05B0F0BDC04602290000034B10B5DD
:10B310001B68002B00D09847FEE7C046F06AFF1F6D
:10B3200007B501A8FFF7F2FF044A05480021121AE9
:10B3300000F04AF8F8F7A0FAFEE7C046F46AFF1FEB
:10B340000444FF1F0000000001B40248844601BC11
:10B35000604700BF3D36FF1F01B40248844601BC70
:10B36000604700BF0D52010001B40248844601BC91
:10B37000604700BF691F000001B40248844601BC59
:10B38000604700BFF938FF1F01B40248844601BC82
:10B39000604700BF993AFF1F01B40248844601BCD0
:10B3A000604700BF6571010001B40248844601BCDA
:10B3B000604700BF7918000001B40248844601BC10
:10B3C000604700BFD91B000001B40248844601BC9D
:10B3D000604700BFB70E000001B40248844601BCBC
:10B3E000604700BFCD4C010001B40248844601BC57
:10B3F000604700BF5952010001B40248844601BCB5
:10B40000604700BF8D1BFF1F01B40248844601BC8A
:10B41000604700BFAD32FF1F01B40248844601BC43
:10B42000604700BF594F010001B40248844601BC87
:10B43000604700BF350E000001B40248844601BCDD
:10B44000604700BFC53AFF1F01B40248844601BCF3
:10B45000604700BFE928000001B40248844601BCEF
:10B46000604700BF091B000001B40248844601BCCC
:10B47000604700BF3D18000001B40248844601BC8B
:10B48000604700BF2D2EFF1F01B40248844601BC57
:10B49000604700BF5147010001B40248844601BC27
:10B4A000604700BFA946010001B40248844601BCC0
:10B4B000604700BF4551010001B40248844601BC09
:10B4C000604700BF0D31FF1F01B40248844601BC34
:10B4D000604700BF1D3AFF1F01B40248844601BC0B
:10B4E000604700BFED3AFF1F01B40248844601BC2B
:10B4F000604700BF3D4B010001B40248844601BCD7
:10B50000604700BFE548000001B40248844601BC22
:10B51000604700BFC94A010001B40248844601BC2B
:10B52000604700BF5D17000001B40248844601BCBB
:10B53000604700BF311B000001B40248844601BCD3
:10B54000604700BF851F000001B40248844601BC6B
:10B55000604700BFA54F010001B40248844601BC0A
:10B56000604700BF8B52010001B40248844601BC11
:10B57000604700BFE538FF1F01B40248844601BCA4
:10B58000604700BFED4A010001B40248844601BC97
:10B59000604700BF5549010001B40248844601BC20
:10B5A000604700BF0534FF1F01B40248844601BC58
:10B5B000604700BF056A000001B40248844601BC30
:10B5C000604700BFB139FF1F01B40248844601BC87
:10B5D000604700BF1147010001B40248844601BC26
:10B5E000604700BF2124000001B40248844601BC2A
:10B5F000604700BFC9A9000001B40248844601BCED
:10B60000604700BF291C000001B40248844601BC09
:10B61000604700BF8530FF1F01B40248844601BC6B
:10B62000604700BF2951010001B40248844601BCB3
:10B63000604700BFDD66010001B40248844601BCDA
:10B64000604700BFB352010001B40248844601BC08
:10B65000604700BFDD52010001B40248844601BCCE
:10B66000604700BFC51D000001B40248844601BC0C
:10B67000604700BFC926000001B40248844601BCEF
:10B68000604700BF8D12000001B40248844601BC2F
:10B69000604700BF4550000001B40248844601BC29
:10B6A000604700BFB54C010001B40248844601BCAC
:10B6B000604700BFADAE000001B40248844601BC43
:10B6C000604700BFC56D010001B40248844601BC5B
:10B6D000604700BF2526000001B40248844601BC33
:10B6E000604700BF6D30FF1F01B40248844601BCB3
:10B6F000604700BF3119FF1F01B40248844601BCF6
:10B70000604700BFE94C010001B40248844601BC17
:10B71000604700BF9DA9000001B40248844601BCF7
:10B72000604700BF434D010001B40248844601BC9C
:10B73000604700BFD949010001B40248844601BCFA
:10B74000604700BF5522000001B40248844601BC96
:10B75000604700BF0519FF1F01B40248844601BCC1
:10B76000604700BF456B010001B40248844601BC3C
:10B77000604700BFEDA5000001B40248844601BC4B
:10B78000604700BF4936FF1F01B40248844601BC30
:10B79000604700BF8552010001B40248844601BCE5
:10B7A000604700BF154D010001B40248844601BC4A
:10B7B000604700BFF30E000001B40248844601BC9C
:10B7C000604700BF1D4B010001B40248844601BC24
:10B7D000604700BF75A9000001B40248844601BC5F
:10B7E000604700BFE117000001B40248844601BC75
:10B7F000604700BFD532FF1F01B40248844601BC38
:10B80000604700BF3D37FF1F01B40248844601BCBA
:10B81000604700BFF137FF1F01B40248844601BCF6
:10B82000604700BF090E000001B40248844601BC15
:10B83000604700BF1D3BFF1F01B40248844601BCA6
:10B84000604700BF2146010001B40248844601BCA4
:10B85000604700BF6DBC000001B40248844601BCD3
:10B86000604700BF5125000001B40248844601BC76
:10B87000604700BF313BFF1F01B40248844601BC52
:10B88000604700BF0124000001B40248844601BCA7
:10B89000604700BF055E000001B40248844601BC59
:10B8A000604700BF156B010001B40248844601BC2B
:10B8B000604700BF090E000001B40248844601BC85
:10B8C000604700BF7139FF1F01B40248844601BCC4
:10B8D000604700BF093BFF1F01B40248844601BC1A
:10B8E000604700BFF94C010001B40248844601BC26
:10B8F000604700BF3555000001B40248844601BCD2
:10B90000604700BF1D4D010001B40248844601BCE0
:10B91000604700BF6D36FF1F01B40248844601BC7A
:10B92000604700BFB14E000001B40248844601BC2C
:10B93000604700BF4D1F000001B40248844601BCAF
:10B94000604700BF3139FF1F01B40248844601BC83
:10B95000604700BF017F000001B40248844601BC7B
:10B96000604700BF014C010001B40248844601BC9D
:10B97000604700BF810E000001B40248844601BC4C
:10B98000604700BFF54E010001B40248844601BC87
:08B99000604700BFC521000063
:10B998000001010302030303040305020602070270
:10B9A800080209000A030B030C020D000E030F0323
:10B9B800100311031303140315001600393C00117A
:10B9C8006D3C00110000000002000000DAB900110F
:10B9D800192A0F180A000000F1590000FD24000080
:10B9E800414601009D7D0011B19D001105720011B5
:10B9F800A17B0011B1530011A5AB00110550001136
:10BA0800493E0011793F00110000000016160000A1
:10BA18000200000024BA0011F4FFF3FFD2FC00007A
:10BA2800B940001100000000000000005475796161
:10BA38000042312E3900303031340067697468753E
:10BA4800622E636F6D2F70767678004254483031DD
:10BA5800000000000200000070BA0011292A282AFC
:10BA6800272A262A252A242A0A180000E204000088
:10BA78007102000078EC000005000000744000002E
:10BA88001027000060F000000400000006640000B9
:10BA9800204E000000000000060000005C4400008A
:10BAA800102700006CEE00000700000005000000F1
:10BAB8001F501D00023CB4000001140019000000D2
:10BAC800810200003031323334353637383941425B
:10BAD8004344454600000000B557001109580011BD
:10BAE8000000000002000000F8BA00116F2A6E2A58
:10BAF8001A18000001A00000000000006410B71D23
:10BB0800C8206E3BAC30D9269041DC76F4516B6B83
:10BB18005861B24D3C7105502083B8ED44930FF045
:10BB2800E8A3D6D68CB361CBB0C2649BD4D2D386FB
:10BB380078E20AA01CF2BDBDFB349B5F8000008048
:10BB48000010000000000000075E00119174001151
:10BB58002B5E001199780011AF5E00116F7800110B
:10BB6800255F001145780011775F00110D7A0011EB
:10BB7800DF5F00110D7A001111600011C779001103
:10BB8800255F0011FD7700119D5F0011A579001157
:10BB9800000000000000000083600011A57900117A
:10BBA800E5600011A9740011052A042A012A002A57
:10BBB80002290328012800280118001800000000A5
:10BBC80000000000000000000000008701010201E1
:10BBD8000201010201020303040103010101010141
:10BBE8000303020103000D000E00100011001300F2
:10BBF8001401070108010A010B011C011D020402BE
:10BC080005020702080219021A021C021D03010399
:10BC1800020317000201000504000807000B0A00D0
:10BC28001716001D1C010201010504010E0D01116A
:10BC380010011413011716011A19020201020B0A46
:10BC4800020E0D0211100214130217160305040345
:10BC58000807030B0A030E0D0001020307090A0B6C
:10BC68000E0F101112141718191A1B1F2021220069
:10BC7800EDA40011A9A500110000000002000000B9
:10BC8800C2BB001100000000D5B200110000000086
:08BC980002000000C0BB001116
:020000041FFFDC
:1000000000000000B13D0011E0B90011DCB90011A1
:100010003461FF1F0000000000000000000000002D
:1000200000000000000000000000000000000000D0
:1000300000000000000000000000000000000000C0
:1000400000000000000000000000000000000000B0
:1000500000000000000000000000000000000000A0
:100060000000000000000000000000000000000090
:100070000000000000000000000000000000000080
:100080000000000000000000000000000000000070
:100090000000000000000000000000000000000060
:1000A0000000000000000000000000000000000050
:1000B0000000000000000000000000000000000040
:1000C0000000000000000000000000000000000030
:1000D0000000000000000000000000000000000020
:1000E0000000000000000000000000000000000010
:1000F0000000000000000000000000000000000000
:1001000000000000000000000000000000000000EF
:1001100000000000000000000000000000000000DF
:1001200000000000000000000000000000000000CF
:1001300000000000000000000000000000000000BF
:1001400000000000000000000000000000000000AF
:10015000000000000000000000000000000000009F
:10016000000000000000000000000000000000008F
:10017000000000000000000000000000000000007F
:10018000000000000000000000000000000000006F
:10019000F932FF1F5931FF1FC16601000000000046
:1001A000000000000000000000000000000000004F
:1001B000000000000000000000000000000000003F
:1001C000000000000000000000000000000000002F
:1001D000000000000000000000000000000000001F
:1001E000000000000000000000000000000000000F
:1001F00000000000000000000000000000000000FF
:1002000000000000000000000000000000000000EE
:1002100000000000000000000000000000000000DE
:1002200000000000000000000000000000000000CE
:1002300000000000000000000000000000000000BE
:1002400000000000000000000000000000000000AE
:10025000000000000000000000000000000000009E
:10026000000000000000000000000000000000008E
:10027000000000000000000000000000000000007E
:10028000000000000000000000000000000000006E
:10029000000000000000000000000000000000005E
:1002A000000000000000000000000000000000004E
:1002B000000000000000000000000000000000003E
:1002C000000000000000000000000000000000002E
:1002D000000000000000000000000000000000001E
:1002E000000000000000000000000000000000000E
:1002F00000000000000000000000000000000000FE
:1003000000000000000000000000000000000000ED
:1003100000000000000000000000000000000000DD
:1003200000000000000000000000000000000000CD
:1003300000000000000000000000000000000000BD
:1003400000000000000000000000000000000000AD
:10035000000000000000000000000000000000009D
:10036000000000000000000000000000000000008D
:1003700021B3001100000000000000000000000098
:10038000000000000000000000000000000000006D
:10039000000000000000000000000000000000005D
:1003A0000000000000000000000000000D1BFF1F07
:1003B000000000000000000000000000000000003D
:1003C000000000000000000000000000000000002D
:1003D000000000000000000000000000000000001D
:1003E000000000000000000000000000000000000D
:1003F00000000000000000000000000000000000FD
:08183800006FFF1F4118FF1FA4
:10184000024981F3088802F09FF90000006FFF1F32
:1018500070B500241E491F4A1F484C6308CA1B0567
:101860001B0DE4188242F9D11C4B80228B630021AE
:1018700009201B4B920519621A4B1B4DDA671B4B53
:10188000DA688243DA609A68194802409A60112047
:10189000296002F08DF8112002F06AF880226B6C4A
:1018A000112093436B64EE23DB006343114A1B0C4E
:1018B00013840122104B9A7201F004FC0F4B1B7829
:1018C000002B04D10E4B1021187802F08DFB70BD57
:1018D000000005408805054000060540FF010000A6
:1018E00000F0004004E100E0003800403CF000401F
:1018F000FFDFFFFF0461FF1FB861FF1FE663FF1FEB
:10190000E461FF1F10B502F0B7F9072804D01228D0
:1019100008D0022808D010BD044A0420136B0133FC
:101920001363F8E70220F6E71420F4E7DC64FF1FF6
:10193000F8B507000C0026002500503630785135E8
:10194000002804D10300287058342370F8BD29788A
:10195000CA00481E8141A3183800A25C5B68C9B266
:10196000FFF7D0FF00280DD12B78DA00A218013341
:1019700050602B703378044A013B3370136A013393
:101980001362D8E70123DFE7DC64FF1F5C234343D6
:10199000074910B5C9180B0058331B78012B05D126
:1019A000FFF7C6FF034A936A0133936210BDC04636
:1019B0001065FF1FDC64FF1F10B502F09DF9064A99
:1019C0000121130010CB4942D967044B136002F088
:1019D000E3F8200010BDC04600E100E01000100058
:1019E00010B5040002F088F9024B1C6002F0D4F834
:1019F00010BDC04600E100E0431E5A425341A02200
:101A0000F0B5D2015B421340154D164A40019B18B8
:101A10002A18127E8BB00191002A1BD01A000832BE
:101A2000D46F0022E6B206AFE4B294420EDC28186E
:101A3000C369002B08D0019902AA117106AA049269
:101A400002AA167303A898470BB0F0BD1978B954D1
:101A50000132EAE71A7D1A7806AB01261A70E6E72A
:101A60009C67FF1F00400040F0B5254B040040017B
:101A7000C25C85B0002A2BD01A18117E002927D00D
:101A8000917E002924D01179022921D11689D78885
:101A9000D168F51BADB22A1C102D00D9102292B2CC
:101AA000BE4217D11818012303710023C269C380F5
:101AB00003819A4206D068460321037301710293A1
:101AC00001A890470820002C00D0192001F0FAFA54
:101AD00005B0F0BD013C65426C41A0256442ED01BA
:101AE0002C40084D1B186419074D0633013A92B279
:101AF000AA42EDD01888461C1E80085C2070F5E7CD
:101B00009C67FF1F00400040FFFF00000F220E4BAC
:101B100010B59868104002380A280BD801F0FEFF73
:101B20000D0A0B0A0A110A0A0A0A060002210020FD
:101B3000FFF762FF10BD0121F9E70020FFF794FFD6
:101B4000F8E7DB6FF6E7C046004000400F220E4B7F
:101B500010B59868104002380A280BD801F0DEFF53
:101B60000E0A0B0A0A120A0A0A0A060002210120BA
:101B7000FFF742FF10BD01210800F9E70120FFF740
:101B800073FFF7E7DB6FF5E70090004013B5334CC8
:101B90002378072B3DD8324B1A78324B002A39D1A3
:101BA0008022196852020A431A60252001F0C0FE03
:101BB00020232D4A11680B43802113606B460422B9
:101BC000C90508680733104228D080210422C905BE
:101BD000C86810422ED080212020C905CA688243DF
:101BE000CA6014221A701A78002A2FD18021C905E0
:101BF000C86820320243CA6014221A701A78002A78
:101C000028D11A4B1A7D22785A601D221A70593237
:101C1000DA6013BD1A6816490A40C5E7086802432E
:101C20000A6014221A701A78002ACED01A78013A63
:101C3000D2B2F7E7C8680243CA6014221A70197852
:101C40004A1ED2B21A700029F9D1C4E71A78013AB3
:101C5000D2B2C7E71A78013AD2B2CEE73C43FF1FAF
:101C60000444FF1F3CF000403443FF1F00200040AD
:101C7000FFFFFEFF564B70B51B68012B03D1554A81
:101C8000936D0133936502F0B7F9534B534A1860D3
:101C9000534B544C1A600123534A1360534A136048
:101CA0002378002B06D006225149524802F00CF846
:101CB00000232370504A514B10681B78C1B2002B8F
:101CC0000ED14F4CC0B223785BB2002B4FDB237890
:101CD00024785BB264B21B0424021B191B18136026
:101CE0000B1C50294ED95023464A47491078DBB285
:101CF000FF2202284BD10868444C454D267890437A
:101D00002A78964254D9227824782E78023B5D10A6
:101D1000A31B6B435201D31A10335B1118430860A5
:101D200002F04AF8031F012B45D83A4B1B78002BD1
:101D300006D0394B1B78002B02D0002002F0CCF8E3
:101D4000A122364B92009978354B4A431B689B1869
:101D5000832292009B181B78033B012B03D8AF20F2
:101D6000400002F051F801222E4BDA8270BD237838
:101D700024785BB264B2FF33FF341B0424021B19C6
:101D80000138ABE7CAB2022AAED20223ACE7086838
:101D9000254C264D267890432A78964208D92278F9
:101DA00024782D78023B5B10641B63435201B2E739
:101DB0002378DBB2B2E70228D5D11D4B1B78013B5B
:101DC000022B03D91B4B1B78022BCCD16C20C8E70C
:101DD0009809FF1FFC0FFF1F2864FF1FFF3F000033
:101DE000141003402C64FF1F0C100340001003402C
:101DF000D50BFF1F7211FF1FB40003408C09FF1F9A
:101E0000680AFF1F490AFF1F94000340460AFF1F8C
:101E1000470AFF1FF908FF1F2209FF1F300DFF1F90
:101E20003409FF1FBC0BFF1F440AFF1F450AFF1F99
:101E30001C09FF1F2309FF1F10B502F07DF80022C7
:101E4000014B1A8010BDC0462464FF1F10B502F07C
:101E500033F8A121054A89009478054A6143126844
:101E6000044B5218528C1A8010BDC046300DFF1F13
:101E70003409FF1F2464FF1F10B50D4B0D4A9978DC
:101E8000A1239B004B431268D218531DD97F0A4BE4
:101E90001B88994209D2441C07D0C82805D0D269B2
:101EA0005B1A5A43054B5343C01801F02DFF10BD78
:101EB000300DFF1F3409FF1F2464FF1F7102000053
:101EC00070B5244D2B68002B28D002F015F82B6834
:101ED000D8402B680400002B27D001F045FE2B686A
:101EE000D8401D4B1D4A9978A1239B004B43126893
:101EF000D118D25C91239B00002A20D0CA5801320D
:101F0000CA50174B17491B680868834214D3D23B49
:101F1000181A012A1AD0144B186070BD01F0ECFF9A
:101F2000124B196801F010FED3E701F01DFE0F4BB4
:101F3000196801F009FED4E70D495B18E8E7CA50BB
:101F40000C4B1B68DB68E418201AE4E7F530FF301F
:101F5000E1E7C0461C08FF1F300DFF1F3409FF1FBB
:101F60009C09FF1F2864FF1FA009FF1F1808FF1FFF
:101F70002DFF3F003064FF1F70B504000D002829BD
:101F800016D10300A433C2881B889B1A0B4A9BB24C
:101F900093420DD906006A3605223100653001F002
:101FA000DBFE002804D13100200001F025FF70BDC8
:101FB0002900200001F0F0FEF9E7C046FE7F000096
:101FC000F8B50500012001F08FFE134CA36AA26A48
:101FD0009342FBD1114E336002F01EF8104903000A
:101FE00008601048426894460F4A17680022BC45B2
:101FF00001D24268BA1A0D4802603268AD18A422B4
:10200000E562606A520302436262094A1278002A5A
:1020100001D00F3B0B60F8BD00F00040340AFF1FF9
:10202000E408FF1F28100040180AFF1F1C0AFF1FAA
:102030001C09FF1F70B580241025E405A3682B43FD
:10204000A36001F011FFA368AB43A36070BD000063
:10205000F7B5160080221C001023D205019191686B
:1020600005000B43936000225A4BD7301A6001F0F1
:102070004BFF9D232A002F009B00EB58CA32012101
:102080000092FC37002B01D00021009A386801F043
:10209000E3FD2900009BCB311A784F4BD3351A60F2
:1020A0004B780A781B0213438A7812041A43CB78C0
:1020B0001B061343494A1BBA13604B790A791B026A
:1020C00013438A7912041A43CB7931001B06134358
:1020D000434A1BBA13606B782A781B021343AA7811
:1020E00012041A43EB781B0613433E4A1BBA1360D3
:1020F000019A330213433C4A13603C4B22001B1BE2
:102100009C4603293DDCB3089A0013005142B21AE1
:10211000032A46D1354AE018511A827840781204D1
:1021200000020243E05C043302430A600022FF2BFA
:102130004BDDF0222E4B12011A600F222D4B1A603C
:102140002D4A1368002BFCD00023224A2749136034
:10215000091B321D0B191B68043A180A23706070A2
:10216000180C1B0EA070E3700434002AF2DC8022ED
:1021700010213B68D20501333B6093688B43936029
:10218000F7BD6346D578981893782D061B042B432A
:10219000157804392B43557804322D022B43036004
:1021A000AFE7022A0AD1114AE05C511AE2185278CC
:1021B000120202430A6004339BB2B7E7012AB5D189
:1021C0000A4A521AE15C1160F5E7084959180A6099
:1021D0000433ACE7000004403C00044038000440F5
:1021E00034000440300004400C000440000104406E
:1021F000040004401000044014000440F7B515002A
:1022000080221C001023D2050091916807000B4327
:1022100093600023654AD730136001F075FE9D235B
:102220003E009B00F9583B00CA363200FC330029BF
:1022300000D07FE0586801F00FFD390032785C4B28
:10224000CB311A604B780A781B0213438A78AC466C
:1022500012041A43CB78281D1B061343554A1BBA98
:1022600013604B790A791B0213438A7912041A43CB
:10227000CB791B061343504A1BBA13604B7A0A7A78
:102280001B0213438A7A12041A43CB7A21001B06DD
:1022900013434A4A1BBA1360009A2B021343484A5D
:1022A00013602200474B1B1B0093009BCE785B18EA
:1022B00001938B7836061B0433430E78043833437E
:1022C0004E78043136023343019E33600328ECDC40
:1022D0000321A808431C9B002940800003292BD11F
:1022E0003849E5185E18A9786D78E35C09042D0279
:1022F000294319433160030008330021FF2B2DDDF2
:10230000314B324919600F21314B196001232749A4
:102310000B60304B19680029FCD006211B680B406C
:10232000042B20D080220020D20593680A318B43F1
:102330009360FEBD01217DE7022908D121495D1886
:10234000E1184978E35C090219432960D3E70129C0
:10235000D3D11C495918E35C0B60CCE71948181815
:1023600001600433CAE7002310490B606346002B69
:102370000CDC3B00FC335A68102101325A60802289
:10238000D205936801208B439360D2E7009B9B1892
:102390001B68190A13705170190C1B0ED37004239B
:1023A0005B4291709C440432E0E7C0460000044068
:1023B0003C00044038000440340004403000044035
:1023C0000C0004400001044004000440080F000019
:1023D000100004401400044070B5061E19D00222FB
:1023E0005A4B9B799343012B13D1594B1A78FF2AEF
:1023F0000FD15A78FF2A0CD19A78FF2A09D1DA78BE
:10240000FF2A06D11A79FF2A03D15B79FF2B00D16D
:1024100099E0504B0C201A78012A08D000224E4D2A
:102420001A7029780B00093B042B01D8212070BDBC
:102430004B1F012BFAD9454CA37B042B00D982E01A
:10244000A279032A00D97EE09A1ED2B2012A02D8CC
:1024500060881F2877D9002E56D0012E73D1A0880E
:102460000128E3D0002907D1581E032803D801F022
:1024700055FB121715122E702978481E032811D803
:102480000025364B1D602823237501F00DFCA84262
:1024900027D0A580CAE702212970EDE70421FBE7D8
:1024A0000321F9E707390129C0D82D490968C96A0C
:1024B0008906BBD52B4908780028B7D1012A01D954
:1024C000002BB3D102230B708021274D26338901C5
:1024D0002878237501F000FC80212878890101F01B
:1024E00083FD0123A380214B1B78002B0AD0FA2205
:1024F00080211F4B92001B8809025A431A4B1878FF
:1025000001F08AFB002092E701F0F6FB2B78A68011
:10251000073B012B03D917482E7001F015FC114B16
:10252000114C1A78002A06D08021002220788901D7
:102530001A7001F0D1FB01F02FFB802120780902F5
:1025400001F0CAFBDEE7122071E7C046A60BFF1FB1
:102550006B09FF1F1A09FF1F1C09FF1F4809FF1FF6
:102560003064FF1F2309FF1F1B09FF1F2109FF1FE5
:102570002C09FF1F0010004010B5002901D001F008
:1025800043FB10BDF7B5604B01919978A1239B00E7
:102590004B435E4A060014681022E418D6235B0001
:1025A000E0583623FF33E35C00279343222B41D1CD
:1025B000574B0F3A1A600760012501F02DFC019B73
:1025C0001880E8235B00E35C002B01D0B34258DDA8
:1025D0000023504FFB70AD33FF33E3581A68002AD5
:1025E00003D09B88DB439B071DD03823FF33E35C7C
:1025F000002B18D09B235B00E35C002B13D1D1335D
:10260000FF33E35CB3420EDAA4235B00E15AE01827
:10261000090A023101F098FC23000122FE33013E39
:1026200001351A87FA70E8235B00E35C002B2AD09F
:10263000A8B2FEBD03683D00002BBED081880430E7
:10264000090A023101F080FCD6235B00E3581F60C9
:10265000B2E72300B133BA00FF33985801378188BD
:102660000430090A023101F06FFCE8235B00E35CEF
:10267000BB42EEDCE822F61AED1800235200A35408
:10268000A6E70027F1E7200001F0FEFB00281FD09D
:10269000002E1DDD7319882647190193B60020000E
:1026A00001F082FA5A308000201840680135818894
:1026B0000430090A023101F047FC200001F094FACD
:1026C000A3590133A351BD4202D0019B9D42E6D1E3
:1026D000114BE35C002BABD095239B00E35C002BFC
:1026E000A6D00E4BE15A0029A2D00D4AA35C994214
:1026F00002D90133A3549BE700231A212000A354DD
:1027000001F0CAFA94E7C046300DFF1F3409FF1FDD
:1027100000140340E010FF1F5A0200007202000084
:102720005E0200000D4970B54A6E0D4CD2038B69F4
:10273000D20BA24206D80B4D0224AA4204D901F0C2
:102740004BFA70BD02246442E21815007E24254035
:102750002242F4D0A3432B438B61F0E700F000400A
:102760000A200000FC1C0000F8B51D4B1D4F1A7814
:10277000002A10D1BA7B002A02D101321A7003E07C
:10278000032AFAD0022AF8D001F08EFA00220120A2
:10279000154B1A70F8BD154B154D1C68154B9E78DE
:1027A00001232B702878C0B200F09EFBBB7B002B6E
:1027B0000BD101F039FCA1239B007343E418832360
:1027C0009B00E41823782B70E4E7032B02D101F07F
:1027D000F3F9F0E70020022BDCD101F0A5FAEAE7DB
:1027E0001C09FF1FA60BFF1F2309FF1F3409FF1F32
:1027F000490AFF1F300DFF1FF0B587B00EAD2F78CF
:102800000FAD2D780593AC46634614000E4D0CAA0F
:1028100012782E7803930D9B009201932200059B62
:10282000029701F011FB2E70012C01D0042C08D16D
:10283000802206498B889343054A1278D2011343BC
:102840008B8007B0F0BDC0461C09FF1F6C11FF1F35
:102850007809FF1F0B001B3B70B504003020E02BF4
:102860000DD81300E025493BFF3B9BB2ED00AB4286
:1028700005D8034B200019825A8201F0DDFB70BDA0
:102880008410FF1F10B501F0B7FB054B00205B68FB
:10289000052B04D9034A5268D20200D4980810BD0F
:1028A00000100040FCE100E070B501F025FA0D4B8E
:1028B0001B68FC33DC691D6AFFF7E4FF641984427E
:1028C00004D2094B01241B68002B07D004220024EA
:1028D000064B1A70064A93690133936101F05CF963
:1028E000200070BD3064FF1F9809FF1F2309FF1FE0
:1028F000FC0FFF1F70B50C4D2B68FC335C6A01F0B8
:10290000FBF9FFF7BFFF2B680025FC339B6AE31838
:10291000834204D2054B1B68AB4200D1051B01F07A
:102920003BF9280070BDC0463064FF1F9809FF1FA7
:10293000D722044B92009B5810B5002B00D098472B
:1029400010BDC0460000FF1F10B501F0CFF8FFF723
:10295000EFFF2749274BCA6D274C1A4084235B00A1
:102960001343CB65254B1B68186A01F0BDF9244B56
:10297000244A1A60244B254A1A60A022244B520094
:102980001A60244B187801F04FF92000224901F019
:10299000F3F90023A3600233A360204B2049236096
:1029A00003232048A36001F0E7F910221E4BFF200B
:1029B0001A60802252031A60802292031A608022D9
:1029C00012041A6001F088FA012001F0D5F8FA200B
:1029D000400001F0F9F9582001F016FA134801F00F
:1029E000E3F9012001F0A8F9072001F0FDF910BD7D
:1029F00000F0004000FEFEFF141000403064FF1F96
:102A0000000003400180063DBC0003403408000084
:102A1000A40003404A0AFF1F71020000C30900001E
:102A2000FFFF3F002810004000E100E0307500008B
:102A3000674E336888331B6883F3088801F054FAC3
:102A4000644A6549136800200B401360634B644A75
:102A50001B68934200D1A6E001F086FA0221614A88
:102A600013688B431360FFF76FFF5F4B5F4C187861
:102A7000C0B201F0A9FA0023A3600233A3605C4B4B
:102A80000120236001F030F90323A36001F00CFA68
:102A9000040001F0B1FA050001F006FA554B186088
:102AA00001F0C2F9544B1968621A531EA14200D2B8
:102AB00013008022D203934201D39B029B0A326807
:102AC000D16AC90700D471E04C491C0C09689BB25B
:102AD0004C4359432402090A641803264849FC322E
:102AE00093680A6847489B1A474A0768126847492B
:102AF0009B18474A9A1833409208DB190A60036012
:102B0000042B03D9013233400A6003600E68414947
:102B1000A619300001F018F83F4F3E493B68C31832
:102B20003B603000019301F067F83C4E30680818B4
:102B300038493060884205D9019B01333B6001F080
:102B40005BF8316001F008FA354B1B78002B0DD093
:102B500001F052FA334B621B196812188A4232D2C2
:102B60004919091B091A304801F006F92F4E337A2A
:102B7000002B0ED001F040FA621BF168121891424E
:102B800024D94919091B091A294801F0F5F800232D
:102B90003372284B83F3088801F0C6F9002001F056
:102BA000E3F901F0E9F901F0DFF95CE7DC019900F4
:102BB0000234641A5900641A09214B438033CB4014
:102BC000A408E41889E7FA218900CCE71A49DBE771
:102BD0003064FF1F1CF00040FFFFC1FF0C0AFF1F05
:102BE000B641210310000040490AFF1F14100040A5
:102BF000C3090000100AFF1F340AFF1F380AFF1F15
:102C0000200AFF1F280AFF1F1C0AFF1F240AFF1F9C
:102C1000C4090000710200006008FF1F2C0AFF1F9A
:102C20001C09FF1FE408FF1F00100040740BFF1F6A
:102C30003C10004000000020DC050000A022054BF5
:102C400092009B5810B5002B01D0984710BD01F0A1
:102C50001BF8FBE70000FF1FA122054B92009B58C9
:102C600010B5002B01D0984710BD01F00DF8FBE71F
:102C70000000FF1FA222054B92009B5810B5002BAD
:102C800001D0984710BD00F0FFFFFBE70000FF1FD9
:102C9000A322054B92009B5810B5002B01D09847FA
:102CA00010BD00F0F1FFFBE70000FF1FA422054B61
:102CB00092009B5810B5002B01D0984710BD00F032
:102CC000E3FFFBE70000FF1F70B501F095F94F4BE4
:102CD000186000F041FF0400C30702D401F0ACF813
:102CE00070BD00224A4B1A604A4B187801380428FC
:102CF00029D800F013FF0320181C2400200000F046
:102D0000DBFF0128ECD0444C2378042B6ED101F07A
:102D10002BF80028E4D001F05FF8582001F074F897
:102D200002232370DCE7200001F0B6F8E9E7200079
:102D300000F082FFE5E7200001F08EF8E1E72000D7
:102D400001F02AF9DDE701F037F80500012808D184
:102D5000324B1B78053B012B03D82000FFF76EFF99
:102D6000D1E72D4B1B78022B01D0052B20D1022D52
:102D700028D12B4B9B7BAB431CD12000FFF76CFF72
:102D8000264B18780128BED16405BCD424492522DD
:102D90004B7B034205D1233A13405A425341263319
:102DA0001A000B7D9342AED9322001F0FDF8AAE75C
:102DB000022D07D1194B1B78052B11D12000FFF7ED
:102DC00059FFDDE7012D0BD1012B03D12000FFF7C7
:102DD0005FFF98E7062B03D12000FFF767FF92E71C
:102DE000200000F051FF022D8DD1C9E7032B04D143
:102DF0000C4B987C00F090FF72E7072B00D06FE738
:102E0000094B987B00F0E0FE6AE7C0469C09FF1F73
:102E10009809FF1F9009FF1F2309FF1F1C09FF1FAF
:102E2000A60BFF1FBC0BFF1FD40BFF1FFA210A4B81
:102E30000A4A49001A640A4A5A500A4A04395A503E
:102E4000094A08319A64094A5A50094A5C315A5071
:102E5000084ADA667047C0460000FF1FF927FF1FC7
:102E6000F528FF1FA928FF1FD923FF1F6927FF1F70
:102E7000791EFF1F4D1EFF1FF7B50B0CFF27012208
:102E8000009300233C001E001D009446019089B26F
:102E900062469A401000084018413618B6B2FF2F1B
:102EA00002D1012E00D19FB2009802401A41AD1804
:102EB000ADB2FF2C02D1012D00D19CB20133102BF9
:102EC000E6D10320012E07D1012D04D1019B24015D
:102ED000E4191C700138FEBD102EFCD10238102DF3
:102EE000F9D00230F7E700008023F7B59C46264B67
:102EF000264F01932649274A274D284C284B022864
:102F00001AD1604638600868264E30408026360365
:102F10003043086001990978002909D11660224AD6
:102F20002A60224A2260E02219689143A03A1BE0FD
:102F30008021C9021160F2E766463E600F68194EB3
:102F40003E408027FF023E430E6001990978002928
:102F50000DD1176001280ED1154A2A60154A22604A
:102F6000E02219689143C03A0A431A60F7BD8021F4
:102F700089021160EEE7E0210F4A02432A600F4AFE
:102F800022601A688A43F0E74B0AFF1FE000034003
:102F9000D80003409000034000000340500003406D
:102FA00040000340FFFFE3FF0280063D804508220A
:102FB0000180063D80660822008006988055082220
:102FC000F8B51E4B80261A680020140034403242A7
:102FD00032D11A681A4F32431A6001223B68063018
:102FE00093433B6000F080FE0122164D2B681E4388
:102FF0002E603B680A2613433B608027BF00124BBC
:103000001B683B4211D1013EF6B2FF2E09D17E2250
:103010000E4B1C682B68E40B1440934323432B6036
:1030200005E0082000F060FEE9E7002EEFD18022E5
:103030002B68600893432B60F8BDC046C4F0004085
:103040005CF0004018F0004068F0004060F0004084
:1030500010B500F0F9FD01215820034A00F0D4FF1B
:10306000FFF7AEFF10BDC046600AFF1F10B5782203
:103070000021034800F0B0FF00F0F6FD002010BD75
:103080002467FF1F70B5040000F036FE00230C20FB
:103090000B4A010059438D18515C00290DD0A14203
:1030A00008D1012300246B7000F086FF00F074FD4E
:1030B000200070BD01330A2BEBD11224F6E7C04685
:1030C0002467FF1F70B5040000F016FE00231900EE
:1030D0001D000D4A1078002806D0A0420CD1557072
:1030E00001310C320A29F5D1002B0AD100F0BCFDC8
:1030F00000F052FD002070BD5078461EB0411B18F4
:10310000EEE700F059FFF3E72467FF1FF7B504006F
:103110000C20002384460E4D019267465F43E85D14
:103120007E19A04212D000280BD10A4B9C46624661
:103130001B7808331370019B70707C557160B3600D
:10314000FEBD01330A2BE8D10320F9E70720F7E79A
:103150002467FF1F2067FF1F8020F8B5484BC0057C
:103160001B68C1248360474BFF251A680123134362
:103170004361454BA4001A68444B40211A60444BFC
:103180001A68444B1A60444B1A59AA431A51C52273
:1031900092009E58AE433143802699509F583F4934
:1031A000F6010F403E439E509E5880273602360A55
:1031B0003043985080201A5900020A4002431A51A5
:1031C00004341A59364E3F04324080263A431A518D
:1031D0001A5936061202120A32431A5108341A5981
:1031E00080260A4002431A51C32292009F58B446D7
:1031F000AF4337439F509F58294E0F4007439F507E
:103200009F58374080263604374380269F509F586A
:1032100036063F023F0A37439F50C0221F59AF4333
:103220003A431A511A591202120A1643C6221E5163
:1032300092009C58AC4365462C439C509C580025FA
:103240000C4020439850C72080001A58154C11405C
:10325000C02212020A431A50134B1B78DB08AB4200
:1032600001DC0020F8BD2378002B06D0A368002BDA
:1032700000D0984701350C34EEE71220F2E7C04643
:103280003843FF1F3443FF1FB0F000401C67FF1F8F
:10329000B4F000401867FF1F00E100E0FF00FFFFEF
:1032A000FFFF00FF2467FF1F2067FF1F030010B50B
:1032B0001F2809D8072200201340072404490A7850
:1032C000A24313430B7010BD00230620F5E7C04650
:1032D0002067FF1F054B06491B780A6805485B07F6
:1032E00002401B0B134300200B6070472067FF1F39
:1032F0001CF00040FFFFC1FF70B50C25FFF7EAFF8F
:103300000A4B1C780A4BE4086543ED18002C01D1E8
:10331000200070BD2B78002B06D06B68002B00D0EE
:103320009847013C0C3DF1E71220F2E72067FF1FB0
:103330001867FF1F1FB5002102220B0001910091A9
:10334000052000F021FD02230B490A681A42FCD136
:1033500020230393039B5A1E0392002BFAD1074AA2
:103360001368002BFCDA0B246C442000012100F0D0
:1033700083FD207804B010BD90C8004000C8004014
:1033800013B504000A4B0193019B002B01D11120BE
:1033900016BDFFF7CFFF23000340044205D00520F0
:1033A00000F0A2FC019B013BEDE71800F0E7C046EE
:1033B000FFFFFF0707B500F09FFC80220821D20520
:1033C000936A0191002B01D10739916202210C4AC5
:1033D00011600199481E01900029FAD10331116052
:1033E000053101910199481E01900029FAD111601F
:1033F000002B02D18022D205936200F0CDFB07BDE5
:1034000000C00040F0B52D4C89B02378002B4FD17F
:10341000FEF7D2FA02232A4F03903A681A42FCD1EF
:1034200020230693069B5A1E0692002BFAD1254EA6
:103430003368002BFCDA0120FFF7A2FF011E02D047
:10344000112009B0F0BD030003220190009005ADEA
:103450009F2000F099FC0321280000F00DFD0223BD
:103460003A681A42FCD120230793079B5A1E079201
:10347000002BFAD13368002BFCDA0120FFF780FF24
:103480000028DDD10398FEF7ABFAAA786B78110417
:103490001B020B4329780B4363601300113B0A495D
:1034A000052B07D801239340A3600B6001232370F1
:1034B0000020C6E780231B03F6E7C0462043FF1F1A
:1034C00090C8004000C800409808FF1F1E4B30B550
:1034D0005A6818781D4B85B0D31859424B410121C9
:1034E0000093002300F0F0FC194B1A4A02259A635E
:1034F00000221A6510325A658022C4219D65164B40
:103500001648D202DA6789004258154B80241A40C7
:1035100080231B0413434350642341200393E40599
:1035200000F006FA402000F003FA6562039D6B1E6E
:103530000393002DFAD103236362FFF73BFFA562DB
:10354000FFF760FF05B030BD2C43FF1F95FFFEF76E
:1035500000C80040050001FF04E100E000E100E0D8
:10356000FFFF00FFF0B585B00700FEF725FA022344
:1035700005002D4C22681A42FCD120230093009BA9
:103580005A1E0092002BFAD1284E3368002BFCDA29
:103590000120FFF7F5FE002803D01124200005B01C
:1035A000F0BD234B2360022322681A42FCD1202362
:1035B0000193019B5A1E0192002BFAD13368002B14
:1035C000FCDA0120FFF7DCFE0028E6D1194B1F6072
:1035D000022322681A42FCD120230293029B5A1E26
:1035E0000292002BFAD13368002BFCDA0120FFF79E
:1035F000C7FE0028D1D1104B2360022322681A4253
:10360000FCD120230393039B5A1E0392002BFAD173
:103610003368002BFCDA0120FFF7B2FE041EBCD198
:103620002800FEF7DDF9B9E790C8004000C8004067
:1036300001000006A8C800400180000110B500206C
:10364000FFF790FF10BD000010B5064B18705960D1
:10365000FFF73CFF00211320034AFFF757FD00202E
:1036600010BDC0462C43FF1FCD34FF1FF0B5040032
:1036700085B003920291FEF79FF9882263035B0BEA
:1036800052051A438023DB059D6A8023274F009251
:10369000BA68002601901B039A420CD9F823260031
:1036A0001B041E401C4206D08022214B52025E6247
:1036B00019680A431A60002D0BD100F01DFB02228D
:1036C0001C4B1A608023DB055A62013A9A6200F0B3
:1036D00063FA0023039A934220D1002D0AD100F00F
:1036E0000BFB144B03221D608023DB055A629D6295
:1036F00000F052FA8023BA681B039A4208D9002EC0
:1037000006D000220A4B0C495A621A680A401A6015
:103710000198FEF765F9002005B0F0BD009A029906
:10372000D2181278CA540133D4E7C0462043FF1F91
:1037300000C8004000C00040FFFFFEFFF0B587B0AA
:10374000029103920400FEF737F9019000F0D4FAD9
:10375000802302250122234EDB0535605D629A62DB
:1037600000F01AFA204F3B682B42FCD1202304932F
:10377000049B5A1E0492002BFAD11C4D2B68002B7F
:10378000FCDA0120FFF7FCFD002802D0112007B071
:10379000F0BD2000039A029900F0F6FB022304001A
:1037A0003A681A42FCD120230593059B5A1E0592C4
:1037B000002BFAD12B68002BFCDA0120FFF7E0FD8B
:1037C000051EE3D100F098FA80230322DB05356063
:1037D0005A629D6200F0E0F90198FEF701F9E0B24B
:1037E000D5E7C04600C0004090C8004000C8004077
:1037F000F0B5802489B00600FEF7DEF8E405A36A80
:1038000002250393029000F077FA0123304F3D60C8
:103810006562A36200F0C0F92E4C23682B42FCD1F4
:1038200020230593059B5A1E0592002BFAD12A4DA1
:103830002B68002BFCDA0120FFF7A2FD002803D043
:103840001124200009B0F0BD244B2360022322681C
:103850001A42FCD120230693069B5A1E0692002B87
:10386000FAD12B68002BFCDA0120FFF789FD021E3C
:10387000E6D11B4B03211E60030001900090202025
:1038800000F082FA022322681A42FCD12023079317
:10389000079B5A1E0792002BFAD12B68002BFCDAEB
:1038A0000320FFF76DFD041ECAD100F025FA802326
:1038B0000322DB053C605A629C6200F06DF9039BB9
:1038C000002B01D1FFF776FD0298FEF789F8B8E7E3
:1038D00000C0004090C8004000C800400100000641
:1038E00094C8004007B5000201910422000A01A912
:1038F000FFF724FF0EBD000073B5050005240B4A39
:10390000A3005B429B1819686B46DE1D3000FFF771
:10391000B3FA022804D133782B55013CEFD276BD9F
:10392000052CFCD00128FAD10230F8E71409001167
:103930001F2807D8012380228340D20591680B43BA
:10394000936070473F2808D80123802220388340A5
:10395000D20551690B435361F3E75F28F1D8012386
:10396000802240388340D205116A0B431362E8E796
:103970001F2807D8012280218240C9058B68934304
:103980008B6070473F2808D8012280212038824070
:10399000C9054B6993434B61F3E75F28F1D80122D6
:1039A000802140388240C9050B6A93430B62E8E7E7
:1039B0001F2810D880230200DB05153A1968012A58
:1039C00006D820229143196019680A431A6070478B
:1039D00001228240F6E73F2811D880230200DB0550
:1039E000353AD968032A06D810229143D960D9689C
:1039F0000A43DA60EBE7012220388240F5E75F28CE
:103A0000E5D842238022181A413B8340D205516AEF
:103A100099435162516A0B435362D8E710B50400D1
:103A2000012813D1A022184992050B685B015B099C
:103A300013430B60154B164A19681140154A0A4387
:103A40001A60402219680A431A6010BD0028FCD190
:103A500001000A2000F060FA21000B2000F05CFA5F
:103A6000C0220A4B920019680A4340211A601A6862
:103A70008A431A60B022044912060B685B015B0995
:103A800013430B60E1E7C04614F000401CF0004017
:103A90007F00FEFF80FD010072B6074A1368013304
:103AA00013600422054B1A600023054A136080222C
:103AB000D2055360FEE7C0467808FF1FC0F0004003
:103AC000C4F0004005490B68002B05D1044A0A6088
:103AD00004490A60044A13607047C046140AFF1F75
:103AE000841E0000380AFF1FC4F000400023034A70
:103AF0001360034A1360034A1360704754F0004098
:103B000040F1004044F1004002B4714649084900C8
:103B1000095649008E4402BC7047C04602B4714643
:103B200049084900095C49008E4402BC7047C04600
:103B300003B47146490840004900095A49008E44BF
:103B400003BC70470000000001B40248844601BC79
:103B5000604700BF090E000001B40248844601BC62
:103B6000604700BFBD0B010001B40248844601BCA0
:103B7000604700BF6D0B010001B40248844601BCE0
:103B8000604700BF6911010001B40248844601BCCE
:103B9000604700BF29B3001101B40248844601BC4C
:103BA000604700BF9DA9000001B40248844601BCE3
:103BB000604700BFD9B0000001B40248844601BC90
:103BC000604700BF75F8000001B40248844601BC9C
:103BD000604700BFC1F7000001B40248844601BC41
:103BE000604700BFD1AE000001B40248844601BC6A
:103BF000604700BF5976010001B40248844601BC09
:103C0000604700BF090E000001B40248844601BCB1
:103C1000604700BFE9D4000001B40248844601BCFB
:103C2000604700BF8B52010001B40248844601BCCA
:103C3000604700BFEDA5000001B40248844601BC06
:103C4000604700BF0534010001B40248844601BC4E
:103C5000604700BFED68010001B40248844601BC22
:103C6000604700BF2144000001B40248844601BC03
:103C7000604700BFADAE000001B40248844601BCFD
:103C8000604700BFE927000001B40248844601BC38
:103C9000604700BFE917010001B40248844601BC37
:103CA000604700BF53B9000001B40248844601BC1C
:103CB000604700BFA9D8000001B40248844601BC97
:103CC000604700BF0134010001B40248844601BCD2
:103CD000604700BFE94C010001B40248844601BCC2
:103CE000604700BFB352010001B40248844601BCE2
:103CF000604700BF0189000001B40248844601BC4E
:103D0000604700BF75A9000001B40248844601BCA9
:103D1000604700BF8937010001B40248844601BCF6
:103D2000604700BF4DF9000001B40248844601BC61
:103D3000604700BF19FA000001B40248844601BC84
:103D4000604700BFE512010001B40248844601BC8F
:103D5000604700BFC1A5000001B40248844601BC11
:103D6000604700BFCD4C010001B40248844601BC4D
:103D7000604700BF01D7000001B40248844601BC7F
:103D8000604700BF2D6C010001B40248844601BCAD
:103D9000604700BF496D010001B40248844601BC80
:103DA000604700BF51B8000001B40248844601BC1E
:103DB000604700BF8D11010001B40248844601BC78
:103DC000604700BFDD0C010001B40248844601BC1D
:103DD000604700BF8512010001B40248844601BC5F
:103DE000604700BF6DF6000001B40248844601BC84
:103DF000604700BFF90D010001B40248844601BCD0
:103E0000604700BF85C1000001B40248844601BC80
:103E1000604700BF7912010001B40248844601BC2A
:103E2000604700BFCD0C010001B40248844601BCCC
:103E3000604700BFC166010001B40248844601BC6E
:103E4000604700BFDD0A010001B40248844601BC9E
:103E5000604700BF9D6A000001B40248844601BC6F
:103E6000604700BFF535010001B40248844601BC3B
:103E7000604700BFDD3F000001B40248844601BC3A
:103E8000604700BF3D71010001B40248844601BC97
:103E9000604700BF71B0000001B40248844601BC15
:103EA000604700BF0934010001B40248844601BCE8
:103EB000604700BF156B010001B40248844601BC95
:103EC000604700BFF9ED000001B40248844601BC20
:103ED000604700BFC56D010001B40248844601BCC3
:103EE000604700BFED6B010001B40248844601BC8D
:103EF000604700BFC9A9000001B40248844601BC64
:103F0000604700BFE90B010001B40248844601BCD0
:103F1000604700BF8944000001B40248844601BCE8
:103F2000604700BF819F001101B40248844601BC74
:103F3000604700BF7997000001B40248844601BC85
:103F4000604700BF8D82000001B40248844601BC76
:103F5000604700BFC115010001B40248844601BC9E
:103F6000604700BFD544010001B40248844601BC4B
:103F7000604700BF016C010001B40248844601BCE7
:103F8000604700BF8552010001B40248844601BC6D
:103F9000604700BF9573010001B40248844601BC2C
:103FA000604700BFF935010001B40248844601BCF6
:103FB000604700BF6137010001B40248844601BC7C
:103FC000604700BF21A9000001B40248844601BC3B
:103FD000604700BF8914010001B40248844601BC57
:103FE000604700BFB70E000001B40248844601BC20
:103FF000604700BF0D52010001B40248844601BC75
:10400000604700BFC95C010001B40248844601BC9E
:10401000604700BF0167010001B40248844601BC4B
:10402000604700BFBD5C010001B40248844601BC8A
:10403000604700BFE9F6000001B40248844601BCB5
:08404000604700BF116E000093
:1040480002000000BEBB001101000000D0B9001141
:1040580002000000BABB0011010000008840FF1FE9
:1040680002000000D8B9001101000000B461FF1F70
:1040780002000000B8BB0011030000002861FF1F08
:104088001200000002000000BEBB00110100000089
:1040980018BA001102000000BABB001101000000AC
:1040A80015BA00110200000022BA00110300000036
:1040B8006361FF1F02000000B8BB0011030000008D
:1040C8007861FF1F02000000BABB00110100000068
:1040D80014BA00110200000020BA00110300000009
:1040E8003961FF1F02000000B8BB00110300000087
:1040F8005A61FF1F02000000BEBB00110100000052
:104108005CBA001102000000BABB001101000000F7
:10411800D141FF1F020000006EBA0011010000002B
:1041280053BA001102000000BABB001101000000E0
:10413800D041FF1F020000006CBA0011010000000E
:104148008061FF1F02000000BABB001101000000DF
:10415800CF41FF1F020000006ABA001101000000F1
:1041680043BA001102000000BABB001101000000B0
:10417800CE41FF1F0200000068BA001101000000D4
:104188003EBA001102000000BABB00110100000095
:10419800CD41FF1F0200000066BA001101000000B7
:1041A80039BA001102000000BABB0011010000007A
:1041B800CC41FF1F0200000064BA0011010000009A
:1041C80034BA0011020202020202000000000000DC
:1041D800161500001D4C0011E14B0011CCBA00115E
:1041E80090011D0018001800FFFF070102030405D5
:1041F80006020106000000000000000000000000A8
:1042080000000000000000000000000000000000A6
:104218000300000002000000BEBB00110100000006
:10422800ECBA001102000000BABB00110100000046
:104238008C42FF1F02000000F6BA001101000000C6
:10424800AE61FF1F02000000B8BB001103000000B0
:104258001864FF1F02000000BABB00110100000033
:104268008C42FF1F02000000F4BA00110100000098
:10427800B061FF1F02000000B8BB0011030000007E
:104288001064FF1F1200000000010000000001116F
:10429800FFFF0000504859360000000000000000F1
:1042A8000B000500F0000000B400002800280028DA
:1042B8003075A000A000A000A00000080008E001E0
:1042C800F000100010001000100010001000500046
:1042D8005000500010001000D0070000000000003F
:1042E8000F0001000500307507001000010081FF74
:1042F80000000000FF00000069710011716F0011DB
:10430800016D0011FFFF0100FF000000859B0011F7
:104318000199001119980011000000000000000028
:1043280000000800040000003B0001085902E001F9
:1043380088212800FF00000002000000BEBB001119
:104348000100000084BC001102000000BABB00118B
:1043580001000000BD43FF1F02000000B6BB0011B2
:1043680001000000DC67FF1F02000000BABB00115B
:1043780001000000BC43FF1F02000000B4BB001195
:1043880001000000BA43FF1F02000000BABB001181
:1043980001000000B843FF1F02000000B2BB00117B
:1043A80001000000B043FF1F180018001D00900115
:1043B800020000030202000002000000BEBB001160
:1043C8000100000098BC001102000000BABB0011F7
:1043D800010000000044FF1F02000000B0BB0011F4
:1043E800000000000000000002000000B8BB00113F
:0A43F80003000000FC67FF1F20FF18
:040000051FFF184180
:00000001FF
